:0200000270008C
:10200000000002205D230700452307004723070047
:10201000492307004B2307004D2307000000000061
:10202000000000000000000000000000B14F0700A9
:102030005123070000000000532307005523070029
:10204000572307005723070057230700572307008C
:10205000572307005723070057230700572307007C
:10206000572307005723070057230700572307006C
:10207000572307005723070057230700572307005C
:1020800085720700572307005723070057230700CF
:102090005723070057230700BDA007005723070059
:1020A000572307005723070057230700572307002C
:1020B000572307005723070000000000000000001E
:1020C000572307005723070057230700572307000C
:1020D000E96B070057230700572307005723070022
:1020E000572307000000000000000000000000006F
:1020F00000000000572307000000000057230700DE
:1021000000000000000000000000000000000000CF
:1021100000000000000000000000000000000000BF
:1021200000000000000000000000000000000000AF
:10213000000000000000000000000000000000009F
:10214000000000000000000000000000000000008F
:10215000000000000000000000000000000000007F
:10216000000000000000000000000000000000006F
:10217000000000000000000000000000000000005F
:10218000000000000000000000000000000000004F
:10219000000000000000000000000000000000003F
:1021A000000000000000000000000000000000002F
:1021B000000000000000000000000000000000001F
:1021C000000000000000000000000000000000000F
:1021D00000000000000000000000000000000000FF
:1021E00000000000000000000000000000000000EF
:1021F00000000000000000000000000000000000DF
:10220000314932480A1A02D0072291438D4630499B
:1022100030480A1A06D00722914381F30988022226
:1022200082F314882C482D492D4A00F03CF82D48A3
:102230002D492E4A00F037F82D482E492E4A00F03D
:1022400032F82E482E492F4A00F02DF82E482F49FB
:102250002F4A00F028F82F482F49304A00F023F881
:102260002F483049304A00F01EF8304830490022EB
:1022700000F024F82F483049002200F01FF82F4AC0
:1022800090471F481F49884205D00268043003B4B4
:10229000904703BCF7E700208646EC46002000216B
:1022A000274A9047FEE7884207D0521A05D00378A4
:1022B00001300B700131013AF9D17047884202D0E8
:1022C00002700130FAE770470000022000F8012098
:1022D0000000022000000220B8DD0700102B0020C3
:1022E000642B0020B8230700B823070024A60700AA
:1022F000B8DD0700102B0020102B002038A70700A6
:1023000038A7070038A7070038A7070038A7070035
:1023100038A7070038A7070038A70700B6DD070071
:102320000CDE0700642B0020642B0020642B0020AF
:1023300084730020847300208473002085230700A9
:102340000D530700FEE7FEE7FEE7FEE7FEE7FEE7C8
:10235000FEE7FEE7FEE7FEE700F002B8FFF7FCBF8E
:102360000F484FF00701884385460E4880470E48C6
:10237000016841F470010160BFF34F8FBFF36F8FAD
:10238000FFF73EBF09480A490A4A884207D0521A55
:1023900005D0037801300B700131013AF9D1704753
:1023A000000002204D73070088ED00E010A7070031
:0823B000E82A0020102B002098
:1023B8007047000007B5044B0093044A402300F01F
:1023C80032F803B05DF804FBD9230700652B002021
:1023D8002DE9F84388461446B2B10F4B0F4E03253A
:1023E800002743F00109224608EB0701002004F00A
:1023F8009DF80744241A48B933782BB14FF47A4032
:10240800C847013D02D13570BDE8F8830123337018
:10241800002CE8D1F8E700BF40A70700642B002094
:10242800704704F0B3B8F0B595B01D461646084697
:102438000C4601F064FD1A9B0D93CDE90865002553
:102448002B46082205A920460A958DF82C500C9594
:1024580001F07CFD079B0293069B03939DF81430C3
:102468008DF8115003F00302012A1DD1BDF8142084
:10247800059DC3F3C203C2F383168DF81030B20072
:1024880008230EA9204601F061FDC5F3952508AB88
:102498000093324602AB0EA9284600F0DFFB204627
:1024A80001F031FD15B0F0BD022AF8D1BDF8165083
:1024B800C3F3C203C5F389158DF810300827082D1A
:1024C8002E4628BF08263B4632460EA9204601F074
:1024D8003DFDAD1B08AB02AA31460EA8374400F0FB
:1024E80021FC002DEBD1DAE708B5FFF79AFF074882
:1024F800042100F01FFB002803DA0549412000F001
:10250800A1FD044B01225A7108BD00BFD0A60700E7
:1025180054A70700102B0020037813F0040216D0EC
:1025280003F00303012B03D0022B09D001207047CD
:102538000A6800880232C0F3831002440A60F5E793
:102548000B684288023303EB92130B60EEE71046E8
:10255800704700002DE9F04FDFF834A187B00F462F
:1025680000230446861C0DF1070015468DF8073038
:1025780000F0FCFCDAF804203A60DAF80830424F40
:1025880003F580639B1AA7F10409A7F10808B34271
:102598001BD30020002D72D004F00F039B0143F0E1
:1025A800050363F30F00DAF80430C3F309020332BA
:1025B80033444AF822009DF80700CAF8043000F0B6
:1025C80005FD012007B0BDE8F08F0121384600F075
:1025D8002AFE484600F042FE404600F03FFEDAF888
:1025E80008000290C0F3090003300AEB800002A93A
:1025F800FFF792FF029B8346C8B9C3F309020AEBAF
:102608008202D16803919A1C0133C3F309030AEBD0
:1026180083030292D86801F00303012B27D0022B11
:1026280008D01A494FF4C27000F00CFD0CE0C3F357
:102638000900D9E7BDF80E30C3F3891303334FEA15
:10264800104B02EB93030293404600F00AFE10B1D0
:10265800029BCAF808305946384600F0E4FDDAF81B
:102668000830DAF8042003F580639B1A8FE7BDF879
:102678000C30C3F383134FEA104B1344E3E7A4056C
:1026880044F006008FE700BF943C0020B9A707007C
:10269800782C0020064B074810B500221A7001F06C
:1026A800E7FB044610B9044801F064FC204610BD5D
:1026B800782C0020A8A607001CA8070030B50A4CF3
:1026C80071B10A4A0A49121BD20800239A4201D161
:1026D800002030BD31F82350854202D00133F5E7A0
:1026E800034654F83300F4E738A60700A8A6070005
:1026F800E82A0020094B013903EBC000032909D857
:10270800DFE801F00A0204060420704700797047E8
:1027180040797047002070470220704738A60700AC
:10272800034BD3E90130C31A58425841704700BFE0
:10273800782C00202DE9F04387B0FFF7F1FF06461B
:10274800002840F0F080794C04F58055A861BFF36B
:102758004F8FA3680293C3F30903033304EB830089
:1027680002A9FFF7D9FE029B10B1AA69002A5DD021
:10277800C3F30902991C013304EB8202C3F3090372
:1027880004EB8303D268DB68049302F00303022B93
:102798000392029155D1BDF80E306548C3F38918EC
:1027A8004746502F28BF502707F1080167F38F13BA
:1027B800C1F30901ADF80E3001F072FB064600289E
:1027C80000F09D8001F09BFB0023082203A93046FE
:1027D80001F0A8FB0299CB43C3F309030133C1F30A
:1027E80009010331B7EB830F4FEA830204EB810140
:1027F80024D95FFA82F90823A7EB0907304601F0CC
:1028080091FBFFB209F108034A4903F0FC033A4679
:10281800304601F087FB029B08F1030803EB98039D
:102828000293AB69002B43D12F6954E062689A4246
:1028380091D8A260304607B0BDE8F08308233A4635
:10284800E6E7012B5BD1BDF80C303948C3F383119F
:10285800062928BF062161F38913023101F00F010F
:102868008900ADF80C3001F01BFB0646002846D065
:1028780001F045FB0023082203A9304601F052FB72
:102888000027BDF80C20C2F38312BB00974203F166
:102898000803C6D202994A1CC1F309010331029206
:1028A80004EB81010422304601F03CFB0137E8E7E4
:1028B800304601F028FBFFF733FF80F00100C6B275
:1028C800B8E7FB685B7923B13B6831461B6838463B
:1028D8009847FB681F68002FF3D1304601F013FBBF
:1028E8000DF107008DF8077000F040FBAB690BB9DC
:1028F800029BA3609DF8070000F068FBDBE72C69EA
:1029080054B90D4B0D480E49C01AC008000440F0D8
:10291800020000F073F8CEE7236820469B689847CA
:10292800E3681C68ECE7002684E700BF782C0020E9
:10293800A8A60700842C002038A6070038A60700A0
:1029480006A807002DE9F34704460F46914601A95A
:10295800012218461E46FFF7FDFDDFF89C8078B37C
:10296800019D0023A81CB34203EB000132D11E488D
:10297800002100F01DFC80F3100A1C4B1C4A4FEA92
:1029880014499B1AB9EBD30F04D31A4940F2A91082
:1029980000F058FB6B1CC3F30903E40008EB830346
:1029A80004F0380449EA0A40C5F3090544F0010473
:1029B800D860033544EA861343EA872348F825306C
:1029C80098F800301BB1FFF7B5FE0028FBD102B024
:1029D800BDE8F087C1F3090108EB810159F823200C
:1029E800CA600133BFE700BF943C0020A8A60700D7
:1029F80038A60700B9A70700782C002000231A463C
:102A0800FFF7A0BF07B50123019201AAFFF79AFFBC
:102A180003B05DF804FB07B5CDE9002302236A463D
:102A2800FFF790FF03B05DF804FB1FB5CDE9012364
:102A3800069B039301AA0323FFF784FF05B05DF803
:102A480004FB1FB5CDE90023069B0293079B039364
:102A58006A460423FFF776FF05B05DF804FB7FB5EF
:102A6800CDE90123089B0393099B04930A9B0593D3
:102A780001AA0523FFF766FF07B05DF804FB000015
:102A88002DE9F7430446D01C8846164601A90022C2
:102A98008008FFF75FFD254D98B3019FB81C019092
:102AA800C0F30900C0F58063B6EB830F00F10300A3
:102AB8004FEA830905EB80002CD83246414607F0DF
:102AC800FFFC1B48002100F073FB80F310007B1C07
:102AD800C3F30903C7F30907220C05EB8303033784
:102AE80042EA0040E400D86004F0380455F8273082
:102AF80044F0020444EA865203F47C131A4345F86E
:102B080027202B781BB1FFF715FE0028FBD103B057
:102B1800BDE8F0834A46414607F0D2FCA6EB09021D
:102B280008EB090105F10C00C9E700BF782C00206B
:102B3800943C002030B50E4C226903460020114613
:102B480029B9D968087142B923610A6030BDC968DA
:102B58000D79854206D00968F2E7D26814680C60DE
:102B68001360F3E701300A28E9D14FF0FF30EDE7B1
:102B7800783C002038B5084B03F5805201251469CC
:102B88001D7004B938BDE3685D71236820465B6831
:102B98009847E3681C68F4E7782C002030B5C388B0
:102BA80085B004460D4633B1144A00921449154ABB
:102BB800284600F001FC217A05291DD0637A4BB123
:102BC800A088FFF797FD104B104953F8202028469E
:102BD80000F0F2FB227A0E4BA08853F822200392D1
:102BE8000021FFF76BFD039A0A490346284605B002
:102BF800BDE8304000F0E0BB05B030BD48A8070094
:102C080030A8070028A80700B8A80700D9D40700EB
:102C1800DCA807004DA8070007B503460846197A3F
:102C2800052911D05B7A2BB1094A0A49019000F0B5
:102C3800C3FB01980849019000F0BEFB019803B05E
:102C48005DF804EB00F0A6BB002AF8D0F2E700BF5D
:102C580048A80700D9D407002DD807002DE9F0436C
:102C680085B01F460C9D002395F80C902B730646E3
:102C78000C46904629463846FFF790FFB8F1060FF4
:102C880009D8DFE808F00412181F2833400031463D
:102C9800284600F091FB002229463846FFF7BCFF82
:102CA80085F80C9005B0BDE8F083226831462846C7
:102CB80000F082FBEFE7D4E900233146284600F014
:102CC8007BFBE8E7A36800933146D4E90023284654
:102CD80000F072FBDFE7E3680193A36800933146D5
:102CE800D4E90023284600F067FBD4E72369029360
:102CF800E3680193A36800933146D4E9002328468A
:102D080000F05AFBC7E76369039323690293E368FA
:102D18000193A36800933146D4E90023284600F0C4
:102D28004BFBB8E708292DE9F74F80460E461746B2
:102D38001C463DD800251B7B257321461046019370
:102D4800FFF72CFFDFF88CA0DFF88CB0AE4232D949
:102D580018F805205946204600F02EFB0135082DAD
:102D6800F4D11B49DFF874A0DFF874B0204600F0F6
:102D780023FB4FF000094E4524D918F809507E2D41
:102D88001ED8284607F060FB002814BF2A462E22CA
:102D98005946204600F010FB09F10109B9F1080F66
:102DA800E9D1012221463846FFF736FF019B2373FC
:102DB80003B0BDE8F08F5146204600F0FDFACDE79C
:102DC8002E22E5E75146204600F0F6FAE4E700BF78
:102DD80061A807005DA8070057A807005FA80700BB
:102DE80063A807004B1C30B5DB00044612F0030053
:102DF8009BB20DD1074D2A601A44074B1A60074B46
:102E08001870074B1870074B1C80074B198030BD92
:102E18000720FCE7383D0020343D0020303D0020ED
:102E2800403D00203C3D00203E3D00202DE9F74379
:102E3800DFF8BC80B8F800308B4206460D461746CE
:102E480047D300240DF107008DF8074000F08EF8F5
:102E5800224B234A23481B78008892F800C08445F7
:102E68005FFA8CF138BF4C1CDBB238BFE4B2A34226
:102E780028D014781178CBB2884286BF0133DBB2F0
:102E8800002313709DF8070000F0A0F84FF6FF73B9
:102E98009C4220D0144B1B6843F8347003EBC409E0
:102EA8009EB195B1114BB8F800001B682A4631460F
:102EB80004FB003007F004FBA9F80450002003B01D
:102EC800BDE8F0834FF6FF74DCE70020A9F80400A2
:102ED800F5E70920F3E70420F1E700BF403D0020B3
:102EE800303D00203E3D0020383D0020343D00208C
:102EF8003C3D002070B5104C104D22782B789A423A
:102F080000D170BD0E480F4A2378126806880E4813
:102F180002EBC301006852F83320898803FB0600DE
:102F280090470A4922780988D3B2914286BF013373
:102F3800DBB200232370E0E7403D0020303D002055
:102F48003C3D0020383D0020343D00203E3D00201F
:102F5800EFF30583C3F308032BB9EFF31480C043E1
:102F680000F00100704701207047000070B504466A
:102F7800FFF7EEFF012803D01049432000F062F864
:102F8800EFF3108672B60E4A9068012398B99360E1
:102F98000C4B0D4DD3F8801029401160C3F88050B8
:102FA800D3F8841051604FF0FF32C3F884202070AA
:102FB80006B962B670BD2370FAE700BFF0A8070033
:102FC800443D002000E100E0FC06FFBD10B50446CA
:102FD800FFF7BEFF012803D00949512000F032F85D
:102FE800084B9A685AB154B9EFF3108172B6064A81
:102FF80018681060586850609C6001B962B610BDCE
:10300800F0A80700443D002000E100E030B53AB1E7
:103018001368DB430A4D0144814204D1D84330BDD3
:103028004FF0FF33F6E710F8012B5340082213F056
:10303800010418BF2C46013A84EA5303F7D1EBE7A1
:103048002083B8ED07B5CDE900016A46002144F2B6
:10305800020002F02DF903B05DF804FB10B561B170
:10306800B2FBF3F403FB1424A4B244B9C0E900147E
:1030780084608281C381204610BD0E20FCE70920B0
:10308800FAE782B050E8022FC188B2EB324F4FF016
:10309800000317BF92B241EA014142EA014104E04C
:1030A8004268B2EB324F08BF012340E80212002AFF
:1030B800E8D18DF807309DF80730002B0CBF1120A0
:1030C800002002B0704737B550E8013F9DB2C4896F
:1030D80025448489A54228BF2D1B0489A54202BF27
:1030E800BFF32F8F002207E0C5EA030540E801542B
:1030F800002CE9D14FF001028DF803200193019AC9
:103108000A609DF8031001F0FF0321B1006810FA6E
:1031180082F003B030BD1846FBE70A884B889A4214
:1031280009D150E8012FC2EA024240E80123002BEE
:10313800F7D1012070470020704737B550E8023FAB
:103148001FFAA3F5C488A54202BFBFF32F8F002240
:103158000DE0C48925448489A54228BF2D1BC3EAF4
:10316800054540E80254002CE8D14FF001028DF8E3
:1031780003200193019A0A609DF8031001F0FF03F0
:1031880021B1006800EB124003B030BD1846FBE7E0
:103198000A884B889A4209D150E8022FC2EA224293
:1031A80040E80223002BF7D1012070470020704728
:1031B80010B5034653E8000F0A4643E8002494F08C
:1031C800000FF7D110BD10B5034653E8000F40EAD1
:1031D800010243E8002494F0000FF6D110BD10B5A9
:1031E800034653E8002F42EA010043E8000494F044
:1031F800000FF6D110BD10B5034653E8000F00EAE2
:10320800010243E8002494F0000FF6D110BD10B578
:10321800034653E8002F02EA010043E8000494F053
:10322800000FF6D110BD10B5034653E8002F02EB8E
:10323800010043E8000494F0000FF6D110BD10B56A
:10324800034653E8002FA2EB010043E8000494F082
:10325800000FF6D110BD0121FFF7B5BF0121FFF71F
:10326800BEBF0021FFF7C7BF0021FFF7D0BF000096
:1032780010B50446002834D003681BB91A49FF204A
:10328800FFF7E0FE636823B917494FF48070FFF732
:10329800D9FEA36823B9144940F20110FFF7D2FE02
:1032A800E36823B910494FF48170FFF7CBFE238AF6
:1032B80023B90D4940F20310FFF7C4FED4E90123F6
:1032C80021689B1ADBB20A60013BDBB2FF2B226844
:1032D80002D10020107110BD1168481C10600B70DD
:1032E800F2E70E20F7E700BF44A9070037B5044608
:1032F80020B913494FF49270FFF7A4FE00250DF191
:1033080007008DF80750FFF731FE226863681168DF
:1033180099420ED9481E106011F8013CE568218ACF
:1033280001FB0355A36811791B1ADBB2994238BF18
:1033380013719DF80700FFF749FE284603B030BD1A
:1033480044A9070037B50C46054620B9104940F294
:103358004710FFF777FE24B90D494FF4A470FFF723
:1033680071FE00230DF107008DF80730FFF7FEFD11
:103378002A681368591C1160E968641A298AB4FB21
:10338800F1F41C709DF80700FFF720FE03B030BD74
:1033980044A9070010B5044618B906493120FFF7BB
:1033A80051FEA2682AB16369216820699847002301
:1033B800A36010BD8AA907000EB433B5059D044665
:1033C80018B911494220FFF73DFE63691BB90E4940
:1033D8004320FFF737FE23681BB90B494420FFF74A
:1033E80031FE63681BB908494520FFF72BFE35B14C
:1033F80006AB01AA29462046019300F079F802B0ED
:10340800BDE8304003B070478AA907000A2938B5DB
:1034180004460D4602D10D21FFF7F8FFA368226884
:10342800591CA160D554D4E901329A4204D32046EC
:10343800BDE83840FFF7AEBF38BD00002DE9F84FB2
:103448009846DDE90A43154682460F460A464FF07C
:103458000109AA420FD2C14538BFC14613F0010B7A
:1034680001D16CB900240126B8F1010F1BD908F16C
:10347800FF386E43F8E709F10109B2FBF5F2E8E716
:103488009B070ED5B8F1000F0CBF30262026A145AA
:10349800E9D2013C31465046FFF7B8FF002CF6D17F
:1034A800E0E72026F3E7B7FBF6F39D42E1D9DFF822
:1034B8003C80B7FBF6F3504618F8031006FB137769
:1034C800FFF7A4FF3346AB42B6FBF5F6F1D2BBF1EA
:1034D800000F02D00CB1A14501D3BDE8F88F20211F
:1034E8005046013CFFF792FFF4E700BF09AA070026
:1034F8002DE9F74F88461746054620B9AF4940F2EF
:103508005220FFF79FFD6B6923B9AC494FF4157042
:10351800FFF798FD2B6823B9A84940F25520FFF71B
:1035280091FD6B6823B9A54940F25620FFF78AFD43
:10353800B8F1000F00F03E8118F8011B49B92B7B48
:10354800002B00F03781284603B0BDE8F04FFFF7A5
:1035580021BF252940F0B780002698F800302D2B90
:10356800424608F1010823D0302B24D02B2B25D03C
:1035780000242A2B02F1010123D13B681A1D1B6884
:103588003A601C440A4613782E2B26D101324FF09C
:10359800000A104610F8011BA1F1300CBCF1090F0C
:1035A8001DD80A2303FB0A13A3F1300A0246F0E7E9
:1035B80046F00106D1E746F00206CEE746F00406DB
:1035C800CBE711F8013CA3F130000928DBD80A2227
:1035D80002FB0434303C0A46CBE74FF0000A12F8ED
:1035E800011B01F0FB0068289046F8D0782909D81B
:1035F8006F290CD8632962D022D8252963D058298D
:1036080000F0888098F80030002B95D197E7703942
:103618000829F7D801A353F821F000BF973707000E
:103628000D3607000D3607002D3707000D36070049
:103638000B3707000D3607000D3607001D3707004A
:10364800642901D06929DDD13A68D2F80090111DAA
:1036580089EAE9723960A2EBE9724FF0010B092A95
:1036680035DCD34538BFD3462CB1B9F1000F01DBA7
:10367800720700D5013CB30702D5BAF1000F03D099
:10368800F00701D44CBB0024B9F1000F2DDAC9F1C1
:1036980000092D212846FFF7B9FE06F00302022A89
:1036A80004D1BAF1000F01D11CBB0024CDE90046BA
:1036B80053460A2249462846FFF7C0FEA2E73B6860
:1036C8001A1D19783A602846FFF7A0FE9AE70A23E0
:1036D8000BF1010BB2FBF3F2C1E7A345D4D22021D1
:1036E8002846013CFFF792FECCE77107D5D52B2180
:1036F800D0E7A345DAD230212846013CFFF786FE01
:10370800D2E73968CDE900460A1D3A6053460A22D5
:103718000968D0E739680A1D3A60CDE90046534682
:103728001022F5E73B681A1D3A6016F00106D3F837
:10373800009024D1B9F1000F03D0484606F03EFFAF
:103748000646B4421DD809F1FF3919F8011F0029AE
:103758003FF458AF2846FFF759FEF6E728460136EA
:10376800FFF754FE19F806100029F7D1A642BFF456
:1037780049AF20212846013CFFF748FEF6E700261E
:10378800F0E720212846013CFFF740FED9E73B68D7
:103798001A1D3A60302128461C68FFF737FE782149
:1037A8002846FFF733FE00220823CDE900322146E0
:1037B800102280E703B0BDE8F08F00BFC6A907005C
:1037C80070B50D461646044618B908495520FFF746
:1037D80039FC1DB905495620FFF734FC2B682560D4
:1037E80031462046BDE87040184700BF19AA0700B7
:1037F8002DE9F0410D4617461E46044618B91849EA
:103808007520FFF71FFC1FB915497620FFF71AFC32
:1038180023681BB912497720FFF714FC1EB9104919
:103828007820FFF70FFCAB0703D00D497B20FFF78B
:1038380009FCE3689D4204D322696B1E334493421A
:1038480003D907497C20FFF7FDFB2368D3F808E07C
:103858003A46334629462046F446BDE8F0416047DB
:1038680019AA07002DE9F041DDF818800E46174621
:103878001D46044618B922498820FFF7E3FB1FB903
:103888001F498920FFF7DEFB23681BB91C498A20E2
:10389800FFF7D8FB45BB1A498B20FFF7D3FBB207CC
:1038A80003D017499120FFF7CDFBBB0703D014497C
:1038B8009220FFF7C7FBE3689E4204D322696B1E80
:1038C8003344934203D90E499320FFF7BBFB236887
:1038D800CDF81880D3F80CE03A462B4631462046FE
:1038E800F446BDE8F041604763685A68B5FBF2F3F7
:1038F80002FB1353002BD2D001498E20CDE700BF25
:1039080019AA07002DE9F0410D4616461F46044640
:1039180018B919499E20FFF795FB23681BB916496A
:103928009F20FFF78FFB1EB91349A020FFF78AFBE2
:1039380063681B68013B2B4203D00F49A320FFF7A4
:1039480081FBE3689D4207D363681A686B1E02FB1C
:1039580006332269934203D90749A520FFF772FB72
:103968002368D3F810E032463B4629462046F44601
:10397800BDE8F041604700BF19AA070070B550B90B
:103988000E4D0F4C0026641B1423B4FBF3F4B44211
:1039980008D1002010E00368002BF1D0BDE870408A
:1039A800DB6918472B6813B901361435EFE7DB6973
:1039B800284698470028F7D070BD00BFE82A0020A5
:1039C800102B0020014B43600020704770AA0700AD
:1039D8000846704700207047024B1868003818BF27
:1039E80001207047503D002008B50248FFF73CFC15
:1039F800002008BD503D002008B510461A4606F0C4
:103A08005FFD002008BD00002DE9F041804686B02A
:103A180011480F4616461D46FFF71DFC0446C8B957
:103A2800AA083146384600F0B3FC0B48FFF71CFCE7
:103A3800D8F8083053B101228DF800200C9A05926D
:103A4800CDE90147CDE9036568469847204606B0A9
:103A5800BDE8F0811124F9E7503D00202DE9F0433D
:103A6800814687B014480E4615469846FFF7F3FB83
:103A78000446F0B90746BD4215D10F48FFF7F4FBDD
:103A8800D9F808305BB102228DF800200022CDE978
:103A98000126CDE90325CDF81480684698472046CD
:103AA80007B0BDE8F08306EB073000F043FC0137B0
:103AB800E1E71124F3E700BF503D002029DF7047FC
:103AC80028DF704770B503689E6886B004460D46C7
:103AD8006EB114220021684606F01BFDA368059309
:103AE800237901952BB1012B0DD06846B04706B05C
:103AF80070BD01238DF8003023690293E3680393B6
:103B080063690493F1E702238DF80030E3681B032F
:103B18000293F5E70846704700207047024B187A71
:103B2800003818BF01207047403F0020034B187A27
:103B38000122B0FA80F05A7440097047403F0020D3
:103B480008B510461A4606F0BBFC002008BD000068
:103B580008B514220021044806F0DBFC0348FFF7EF
:103B680090FA002008BD00BF403F0020303F0020F1
:103B780010B5094C094B43602046FFF76CFB48B968
:103B880006F07EFA064920741C2306484FF4EE72AC
:103B9800FFF764FA002010BD403F00209CAA0700F0
:103BA800543D0020303F002038B5224D224C2B7A5E
:103BB8003BB922492248FFF7C0FA206008B968607B
:103BC80038BD022324682B72237973B1012B22D0CC
:103BD80020460321FFF776FF00232B726B601749FD
:103BE8001748BDE83840FFF7D3BAD4E90523D21AFD
:103BF800142AD4E9031028BF14229208012A38BFD6
:103C0800012219441844FFF759FF50B11128DFD198
:103C180001232B72D4E7D4E903031844FFF750FFBC
:103C2800F3E72B7C002BCBD1BDE83840022000F015
:103C380009B800BF403F0020583F0020543F0020F3
:103C4800303F002038B5224C237A002B3FD0022B7E
:103C580009D103282ED01F4B00221B68E2601A7975
:103C68003AB1012A20D0637C6BBBBDE83840FFF72E
:103C78009BBFD3E905128D1A142D94BF5219143223
:103C88009A619142EFD102284FF0000308BF19460C
:103C98002372104B18BF0D211868FFF713FF0E4948
:103CA8000E48FFF775FADEE71A6901321A615B6997
:103CB8009A42E7E7E3680133082B01D8E360D2E7CB
:103CC8000023E360DFE7BDE8384006F0C9B938BD36
:103CD800403F0020583F0020543F0020303F002044
:103CE800831E012B01D8FFF7ADBF704700F0FD031D
:103CF800012B08D1044B00225A74421E50425041F5
:103D08001874FFF751BF7047403F002010B5064CAC
:103D1800201DFFF7A0FA28B9637C1BB9BDE8104045
:103D2800FFF742BF10BD00BF403F00202DE9F3411F
:103D380080460D46104801A916461F46FFF7C3F9ED
:103D48000446B0B118220021043006F0E2FB2D0B26
:103D58000123237101A90848C4F80080A760E56021
:103D68006661FFF7DAF9FFF7D1FF002002B0BDE87E
:103D7800F0810420FAE700BF303F00202DE9F3412D
:103D880080460F460F4801A916461D46FFF79BF9C6
:103D98000446A8B118220021043006F0BAFB089B9B
:103DA800A36001A9C4E903670648C4F800806561F7
:103DB800FFF7B3F9FFF7AAFF002002B0BDE8F081D2
:103DC8000420FAE7303F00202DE9F74F99469DF887
:103DD8003030009388469346064618B92349B620E2
:103DE800FFF730F9F28871794A43043A4A4505D811
:103DF8001E490192C420FFF725F9019ADBF80070EB
:103E0800B6F806A007EB0901914209F1040488BF3E
:103E1800A2EB0907B4FBFAF5CBF800700AFB1544CE
:103E280045B9AAEB040BBB4528BFBB462FB903B065
:103E3800BDE8F08F3668013DF2E7009B043408EBDB
:103E4800050034445A466BB12146A7EB0B0706F030
:103E580037FBBA455D443668D3464FF0000428BFA7
:103E6800BB46E3E701462046EFE700BFC8AA0700C4
:103E7800FFF7FEB9F8B546790146721E05460023DC
:103E880093422D6803D30024A64202D8F8BD01331B
:103E9800F6E70F682846FFF755FA01343946F3E785
:103EA8002DE9F843068ACD1C0746FFF71FFA043EA2
:103EB80035440446B5FBF6F5F0B14FF48073EDB226
:103EC8008380C680013D076081464FF00008A84501
:103ED80012D23846FFF70AFA064648B16379013329
:103EE800637108F10108C9F8000007608146EEE730
:103EF8002046FFF7BFFF34462046BDE8F88301217E
:103F08000430FFF790B910B5012104460430FFF7DB
:103F180096F9C0B220B92046BDE81040FFF7AABF05
:103F280010BD00001FB5144603920022009203AA98
:103F3800FFF74AFF039BA34203D00349F620FFF78C
:103F480081F804B010BD00BFC8AA07001FB5144609
:103F580003920122009203AAFFF736FF039BA342B4
:103F680004D003494FF48070FFF76CF804B010BD1B
:103F7800C8AA0700836800225A60C3E904229A602D
:103F8800DA601A607047000038B50D46044618B963
:103F980009495020FFF756F81DB907495120FFF786
:103FA80051F82B686A686360934208BF0023256054
:103FB80008BF636038BD00BF0EAB070010B50446EC
:103FC80018B90B496320FFF73DF823681BB9084966
:103FD8006420FFF737F8636843B122689168526834
:103FE8000B449342636004BF0023636010BD00BFAD
:103FF8000EAB070010B50D49A1F59472914201D896
:1040080000200FE08C1AE30F03EBE4035B1002EBD4
:10401800C30452F83330834205D802D204F10802AF
:10402800ECE7606810BD2146E8E700BF64B0070010
:1040380008B5FFF7DFFF024B002808BF184608BD88
:1040480027AF07002DE9F04FC9B008AA01F14005D4
:1040580014464B780E781B0443EA0663CE78334344
:104068008E78043143EA06238D4244F8043BF0D1AC
:104078001024916B16464FEAF14383EA714383EAB1
:104088009123716A366852F8045F31440B444FEA51
:10409800B54181EAF51181EAD50101340B44402C80
:1040A800D363E6D1D0E914E30093836D0193C36D24
:1040B8000293036E0393436E0493836E0593C36E5A
:1040C8000693DDE9057BDDE9031CDDE901592B4B8E
:1040D800009E079374464FF00008079B53F8042B83
:1040E80007934FEAF12383EAB11383EA716A08ABB5
:1040F80053F828301A440AEB020327EA010A01EAB6
:104108000C028AEA02021A444FEA743A86EA050364
:104118005A4423408AEAB40A06EA050B83EA0B0BE1
:104128008AEAB45A08F10108DA44B8F1400F02EB00
:104138000903BB465244A94619D172440265009A44
:1041480022444265019A32448265029A2A44C26531
:10415800039A1A44049B02660B444366059B634416
:104168008366069B3B44C36649B0BDE8F08F67464B
:1041780035468C46264619461446AEE764B0070015
:1041880030B5E0B10F4A104900240025C0E91245B6
:10419800C0E914120D4C0E4A0E4DC0E916420E4AE3
:1041A800C0E918520D4A826602F17452A2F5230240
:1041B8000023A2F692420364C266184630BD0E2060
:1041C800FCE700BF85AE67BB67E6096A72F36E3C21
:1041D8003AF54FA57F520E518C68059BABD9831FCA
:1041E80070B5F0B1DAB900201CE00C468D18002635
:1041F800AC42F8D0036C14F8012BC2540133402BA5
:104208000364F5D10146FFF71DFFD0E9123213F51B
:10421800007342F10002C0E912320664E8E700299F
:10422800E3D10E2070BD70B50D4616460446002831
:1042380076D0002974D0036C8022591C372BE254A5
:1042480008443FD8C3F13702002106F062F9D4E9E7
:104258001223216C0820E1FB0023C4E9122312BABF
:10426800E26323FA00F284F83B3084F83A201A0C0F
:104278001B0E214684F8392084F838302046FFF791
:10428800E1FE691E6EB30023E26EDA4001F8012FE9
:10429800A26EDA400A71626EDA400A72226EDA4061
:1042A8000A73E26DDA400A74A26DDA400A75626D2B
:1042B800DA400A76226DDA400833202B0A77E3D1F8
:1042C800002070BD4029C3F13F024FF0000188BFB4
:1042D800002206F01EF921462046FFF7B3FE3822D9
:1042E800B2E71823226DDA4001F8012F626DDA4037
:1042F8000A71A26DDA400A72E26DDA400A73226E20
:10430800DA400A74626EDA400A75A26EDA400A76FA
:10431800E26EDA40083B13F1080F0A77E2D1CFE7E3
:104328000E20CEE7024AD2F80034002BFBD07047AB
:1043380000E001400A4908B50223C1F80435BFF37B
:104348006F8FBFF34F8FC1F80805FFF7EBFF00230E
:10435800C1F80435BFF36F8FBFF34F8F08BD00BF9F
:1043680000E0014010B5094C0123C4F80435BFF33F
:104378006F8FBFF34F8F0160FFF7D4FF0023C4F89E
:104388000435BFF36F8FBFF34F8F10BD00E00140BE
:1043980070B50E4E01231546C6F80435BFF36F8F6E
:1043A800BFF34F8F0024AC4207D10023C6F8043571
:1043B800BFF36F8FBFF34F8F70BD51F8243040F8B3
:1043C8002430FFF7AFFF0134EDE700BF00E0014004
:1043D80043689B68184708B5436808305A7900F065
:1043E80007FF002008BD2DE9F0410C469CB00846A7
:1043F8001F460392FFF7ECFFD4F80480039998F85E
:104408000550BD4228BF3D4606462A4604A800F08E
:10441800D3FE98F8052022990CA800F0E9FE009632
:104428000CAB2A4604A904F1080001F099FE002803
:1044380048F2425018BF00201CB0BDE8F0810023AC
:10444800C0E902328B881A44B1F9063002611A4475
:10445800C0E9001142610888003818BF0120704780
:104468004268118838B50346002937D0148A02F10A
:10447800100141602CB9C2680168FFF7E0FF2046CF
:1044880038BD9078118900F03005302D14D1947C16
:1044980004F03004302C1BD190881969091A19616D
:1044A8000021908AB2F9162008441969014419615B
:1044B800114459610120E3E700F0F004202C07D1F2
:1044C80050894143002DECD1986801309860E8E7A5
:1044D80000F0C000802808BF0421F3E70846CFE7B2
:1044E80070B5466804460D4663681A88AA4204D126
:1044F8009B7803F00F03082B07D12046FFF7B0FF86
:104508006368B342F0D1002070BD0120FCE7436826
:104518001A44426011B101399A4201D10120704711
:1045280013F8010B01F8010FF6E770B54568AA7892
:1045380002F00F06082E86B003461FD103691C68D7
:1045480000260CB906B070BD236862689D682673A2
:1045580029466846FFF773FF6368049304F10C0368
:104568000593AB7803F0C003802B08BF231D684672
:1045780008BF0493FFF7D9FFA468E2E712F0C0016F
:1045880022D102F0300010280CD15A691170072E80
:10459800EC6818690BD10146204606B0BDE87040AA
:1045A80000F01AB89006F2D55B691980CAE72A8923
:1045B800214624B106B0BDE8704005F081BF06B0C1
:1045C800BDE8704005F0A5BF8029BBD10069002176
:1045D80092060160B6D5E7E77FB50A460146684608
:1045E800FFF72DFF30B16846FFF79FFF6846FFF7DA
:1045F80037FFF7E707B05DF804FB836810B504469A
:104608000BB9002010BD0368012298470028F8D094
:10461800A368013BA360F5E72DE9F3410F460DF1CF
:1046280007018046FFF7E9FF054620B9002528461F
:1046380002B0BDE8F0819DF907309DF80740002BD6
:1046480013DA04F07F0407260DF107014046FFF74F
:10465800D4FF0028EAD09DF8072002F07F03B3407A
:104668001C43130606F1070601D43C60DFE7232E3E
:10467800EAD1DBE730B5044685B01546A9B902682A
:10468800114B9A4211D0102D06D82A466946204669
:10469800FFF7F0FF05B030BD102269462046FFF74E
:1046A800E9FF0028F6D0103DEDE7A368AB4201D240
:1046B8000020EFE723682A46204698470028F7D0CD
:1046C800A268521BA260E5E717450700F7B50E463A
:1046D80001A907461546FFF79FFFA0B1019A511C93
:1046E8004FF0000404D2B37803F0C003802B01D14B
:1046F800204608E033898B42FAD329463846FFF72B
:10470800B9FF019BEC5403B0F0BD73B50D4601A988
:1047180006461446FFF780FF98B1019AB2F5803F2C
:1047280011D2AB7803F0C003802B02F102010AD04A
:104738002B898B4207D32146304621F8022BFFF7FD
:1047480099FF02B070BD0020FBE7000010B5034CD4
:1047580082600022C0E90041C26010BD1745070011
:104768002DE9F341002580460E462F462C460DF1D3
:1047780007014046FFF741FFC0B19DF807C0A4F10B
:1047880020030CF07F02C4F1200102FA03F322FA9D
:1047980001F10B43A2401CF0800F45EA020547EAED
:1047A800030704F1070404D1C6E9005702B0BDE8C5
:1047B800F081462CDBD10020F8E737B50D46694675
:1047C8001446FFF7CDFF70B12B89082B0DD1DDE919
:1047D8000032C4E90032DDE90001914208BF984285
:1047E8000CBF0120002003B030BD042B03D1009B77
:1047F80023600022EFE7022B03D1009B23809BB2AA
:10480800F7E7012B04D1009B237003F0FF03F0E7C7
:104818000020E8E737B50D4669461446FFF7A0FFC4
:1048280030B12B89082BDDE9001203D1C4E900124D
:1048380003B030BD042B4FEAE17009D121600B466B
:104848000246824208BF8B420CBF01200020EFE7DE
:10485800022B03D10BB22380DA17F2E7012B02D126
:104868004BB22370F8E70020E2E7F7B51F460023B4
:104878003B700D460B70136001A904461646FFF7FE
:10488800CBFE30B9A36813B901233B70002003B0F5
:10489800F0BD019C002CF7D0E30804F00704336056
:1048A8002C70F4E713B50446052925D8DFE801F094
:1048B800030F17242422012201A92046FFF7DAFE5C
:1048C80018B19DF90430002BF5DB02B010BD0822A9
:1048D8000021204602B0BDE81040FFF7CBBE01A979
:1048E800FFF79AFE0028F0D0019A00212046FFF732
:1048F800C1FEEAE70422EBE70020E6E773B50D46C0
:1049080001A90446FFF788FE064618B90026304676
:1049180002B070BD94E80F0085E80F0001998A4243
:10492800F4D3A960A3685B1AA360F0E72DE9F0430C
:104938005668B37813F0C00489B007468C4615460C
:1049480003D0402C69D000240CE003F00F0260492A
:1049580003F03003202B51F8228025D006D8E3B18C
:10496800102B17D0204609B0BDE8F083302BF9D1C1
:104978006B6931881980072A09D12146328928694B
:1049880005F0C7FD6B682969D868FFF725FE2A6915
:10499800696840E06B6901221A702A69314643460A
:1049A80009B0BDE8F0431847BCF1020FD5F81490E0
:1049B80024D1042A22D804A9FFF7A0FF044600281E
:1049C800C1D0069B2BB16968B9F800304A899A4270
:1049D80005D8059B7B60069B002BC3D0B3E70889ED
:1049E8002A6903FB002204A8C04728B1B9F800309F
:1049F8000133A9F80030E4E70446EAE7B9F80030E3
:104A080072899A429FD931892A69581C03FB01226D
:104A1800A9F8000031463846C1E7D2F8108046466A
:104A280056F8043B23B909B0BDE8F043FFF73ABF95
:104A3800022914D104A9FFF761FF002883D0D8F810
:104A480000306968324604A89847044600283FF4B5
:104A58007AAF069B002BF2D1059B7B6082E7012988
:104A680026D005292CD000297FF46DAF0C460DF116
:104A7800040901340B2C3FF466AF0122494638463D
:104A8800FFF7F8FD00283FF45EAF19F9013B002B52
:104A9800EFDB104B049301ABCDE9053400230793FA
:104AA8006968D8F80030324604A89847044659E7A0
:104AB800082201A9FFF7DEFD08240028E9D142E712
:104AC80004220DEB0201FFF7D5FD0424F5E700BF32
:104AD80070B10700174507002DE9F04F91B0044663
:104AE800002604A8CDE90266FFF7A9FCA3683BBB32
:104AF800DDE9053404A89D78FFF7B2FC0028F7D15A
:104B080015F0300F03D1059B1B8803B10134002C2D
:104B180000F0A980630902A90022934240F09C801A
:104B280010AA02EB830304F01F0453F8383CC4F1C5
:104B380020044FF0FF30E040C31A584258410DE0BE
:104B48000DF1030301AA0DF102012046FFF78DFEC6
:104B580038B99DF80330002BCAD1002011B0BDE848
:104B6800F08F019904A8FFF7BBFC002850D1019BE6
:104B7800B3427DD3059D059A937803F00F03082B64
:104B88007FD004A8FFF76CFC059B9D42F3D14FF042
:104B9800FF36019FB7426BD3089B9DF802A0D4F85B
:104BA80008801D684FF00109A368002D5DD0984565
:104BB8009CD12B68D3F800B0BBF1000F08D0534646
:104BC8003A4629462046D8470028C6D0AD68EBE7C4
:104BD800D3F808B0BBF800309F42F7D16A6859464D
:104BE8000AA8FFF72CFC6B680E9305F10C030F93D2
:104BF8009BF8023003F0C003802B04BF2B1D0E93DB
:104C08000AAA85F80C9051462046FFF78FFEDBE78D
:104C1800059B9B7813F0300F0FD1069A3F2A0CD8CA
:104C2800510910AB03EB810102F01F0201239340ED
:104C380051F8382C134341F8383CE5682DB19DF8FC
:104C48000220019904AB2046A8479DF8021004AA47
:104C58002046FFF76BFE10E051F8045B01357FF446
:104C68007DAF013259E7012078E798457FF43EAFE0
:104C78009DF802102046FFF715FE00287FF436AF96
:104C88006BE7168885E737B50C460546114620467A
:104C98000192FFF7A1FC019A2146284603B0BDE81E
:104CA8003040FFF719BF70B586B0CE6801920C4648
:104CB80002A90546FFF722FE68B1E06858B1A3785B
:104CC800019A03F03003202B314602A805D1FFF7E3
:104CD800DAFF039B6B6006B070BDFFF7FDFEF8E7D7
:104CE80013B50C466946FFF73BFD60B1DDE90013DB
:104CF8004A0842EAC372C9074FEA530344BFD24382
:104D0800DB43C4E9002302B010BD37B50D46694640
:104D18001446FFF7E5FF70B12B89082B0DD1DDE9AB
:104D28000032C4E90032DDE90001914208BF98422F
:104D38000CBF0120002003B030BD042B03D1009B21
:104D48002360DA17EFE7022B03D1BDF90030238087
:104D5800F7E7012B03D19DF900302370F1E700201C
:104D6800E9E713B504220C460DEB0201FFF782FCBC
:104D780008B1019B236002B010BD1146FFF7F1BFD7
:104D880013B508220C466946FFF774FC18B1DDE933
:104D98000023C4E9002302B010BD1146FFF7F0BF9D
:104DA8000268530910B5044618D0012B40F2FF33AE
:104DB80018BF002302F01F02D340DB0704D40949BF
:104DC8004FF4F670FEF73EF923681F2B83BF03F0FC
:104DD8001F03054823604FF0A04010BD4FF0FF337C
:104DE800E8E700BF94B1070000030050032813B59B
:104DF800044603D908494120FEF724F9074B01A8C6
:104E08001B5D0193FFF7CCFF019A01239340C0F883
:104E18000C3502B010BD00BFBFB10700FBB10700E1
:104E2800032813B5044603D908494720FEF70AF9B1
:104E3800074B01A81B5D0193FFF7B2FF019A0123FD
:104E48009340C0F8083502B010BD00BFBFB10700DD
:104E5800FBB1070008B50020FFF7E2FF0120FFF7CC
:104E6800DFFF0220FFF7DCFFBDE808400320FFF763
:104E7800D7BF0000F7B5C207044612D5134E002568
:104E8800032716F8013B019301A8FFF789FF019B4F
:104E9800013503F5E073042D40F82370F1D1FFF7D5
:104EA800D9FFA30710D50A4D00240C2615F8013B9D
:104EB800019301A8FFF774FF019B013403F5E07328
:104EC800042C40F82360F1D103B0F0BDFBB107001A
:104ED800F7B1070038B1054B0360054B4360012368
:104EE8000372002070470E20704700BF234F070051
:104EF800FD4E070069B10B78022B0CD1022804D0B3
:104F0800032814BF08201120704703230B700020CA
:104F180070470E2070470820704710B50C4681B1C5
:104F28000B78012B06D00ED9033B012B94BF082028
:104F3800112010BD03F0BEFE0028FAD10223237011
:104F4800F7E70E20F5E70820F3E7000070B5144BEB
:104F5800144A0C21D21AB2FBF1F2816911F8025CF1
:104F6800044635B900690021914205D10123236027
:104F78000EE04FF0FF30F6E71E68AE420CD1461C3B
:104F880007D19D68D4E90001D4E90223A84720602D
:104F980070BD5E688642F4D001310C33E4E700BF8F
:104FA8002CA6070038A607001EF0040F0CBFEFF36D
:104FB8000880EFF30980FFF7C9BF00BF28B139B1F6
:104FC8000023C1E900301846704748F21050704776
:104FD80048F21350704730B1036848F240508B4292
:104FE80008BF0020704748F21050704728B148F2B7
:104FF8001150914208BF0020704748F21050704786
:1050080070B506460C461D46FFF7D8FF50B9B37970
:105018004AB1AB420AD111462046FFF7DCF908B97C
:10502800044B236070BD48F21050FBE748F2115062
:10503800F8E700BF7052464D2DE9F0470C4606468A
:105048000F492046DDE9088915461F46FFF7C3FFCB
:10505800A0B963685A79494652004046FFF7C6FF2F
:1050680060B94DB1CDF820803B462A4621463046EE
:10507800BDE8F047FFF7B7B948F21050BDE8F08730
:105088007052464D10B5044638B149B10B684160BD
:10509800984708B9044B236010BD48F20150FBE75C
:1050A80048F21050F8E700BF6E524648F0B4134675
:1050B80048B10768094EB7420AD161B12AB14368BD
:1050C800F0BC5B68184748F201531846F0BC7047BB
:1050D80048F20253F9E748F21053F6E76E52464891
:1050E800F0B460B107680C4EB7420CD171B1436897
:1050F8001568DC68A5420CD3F0BC9B68184748F2D9
:105108000150F0BC704748F20250FAE748F21350D9
:10511800F7E748F21450F4E76E524648F7B50446EC
:10512800DDE9086715460193FFF7ACFF68B9019AF6
:1051380029462046FFF7BAFF38B93A463146204695
:1051480003B0BDE8F040FFF7CBBF03B0F0BD0000EF
:10515800F8B50A4F0A4C0B4EE41B0123E4083370E0
:105168000025A54203D1022333700020F8BD57F86B
:10517800353098470028F9D10135F2E724A6070011
:1051880024A607005C3F002038B50D46044618B930
:1051980008493320FDF756FF691E21442046814205
:1051A80000D238BD03780A7800F8012B01F80139DC
:1051B800F5E700BFFFB1070070B50D461446064677
:1051C80018B90A494520FDF73DFF1DB90749462092
:1051D800FDF738FF621E3244013DB24200D270BD75
:1051E80015F8013F02F80139F7E700BFFFB10700E2
:1051F80070B5164604460D46FFF7DEFF3246A9197C
:10520800A019BDE87040FFF7D7BF38B50D46044672
:10521800FFF7BAFF29466019BDE83840FFF7B4BF69
:1052280008B507281BD8DFE800F004121A1A1A0478
:105238001A040120FFF71EFE0020FFF7D7FD01200A
:10524800FFF7D4FDBDE808400220FFF7E9BD0120C3
:10525800FFF7E6FDBDE808400220FFF7C7BD08BD1F
:1052680008B5FDF787FCFDF765FA0028FBD10D4D61
:10527800642445F001054FF47A40A847013CFAD16F
:10528800094BD3F8F020D20700D500BEBFF34F8FEB
:10529800D968064A01F4E0610A43DA60BFF34F8F28
:1052A80000BFFDE710B3070000ED00E00400FA05B9
:1052B80007B50B46064C07490092641AE408240413
:1052C8000246054944F00100FDF7AFFBFFF7C8FFB0
:1052D80038A6070038A607008CB2070008B50246B2
:1052E800054B064806491B1ADB081B0443F001005E
:1052F800FDF788FBFFF7B4FF38A6070038A60700BC
:10530800C3B2070010B501F06FFF4FF480510020C1
:1053180001F050FB08B1FFF7E1FF1748C0F5FC2189
:1053280001F048FB01460028F5D11448144CFDF75C
:10533800B1F9FDF7D9F8134B1349E41AE40824042A
:1053480044F00300FDF75AFB00F05CF800F06EF83B
:105358000E4801F0CDF90028DDD1FDF7EBF9002862
:10536800FBD10B4944F00100FDF748FBFDF7E2F9DA
:105378000028FBD1CFE700BF00200700296D0700F8
:1053880038A6070038A60700DEB207002952070032
:10539800EAB20700436810B45BB11548154B1649CB
:1053A8005DF8044BC01AC008000440F00300FDF784
:1053B80025BB0378012B04D0022B10D05DF8044BD9
:1053C80070470C4B0A4C02690C49E41AE4088368DC
:1053D800240444F003005DF8044BFDF71CBB054BA7
:1053E800034C02690649E41AE40883682404F0E7D8
:1053F80038A6070038A6070016B3070057B30700FA
:105408008BB3070008B5064B064907481960002208
:10541800FEF7D6F918B1BDE80840FFF75FBF08BD31
:10542800703F0020A8AA0700E82A002030B591B0F4
:1054380040220021684605F06CF8174840236A4668
:105448004FF4DC21FEF7D4F908B1FFF747FF124CFF
:105458002046FEF793FA0028FAD1104C6B4604ADAB
:105468001A4603CAAA4220606160134604F1080480
:10547800F6D10A4805F0A2F802280BD8074A07AC6B
:105488000BAD234603CBAB42106051601C4602F1C2
:105498000802F6D111B030BDE82A00205D3F002097
:1054A8008B1802448B4200D1704713F8010D02F8A3
:1054B800010DF7E700000000C3F10803DB0070B539
:1054C8000133002403A500BF5B1920C940CAAD19E8
:1054D80020C0184720C940CA754120C020C940CA09
:1054E800754120C020C940CA754120C020C940CAA2
:1054F800754120C020C940CA754120C020C940CA92
:10550800754120C020C940CA754120C06441204669
:1055180070BD00BF00000000C3F10803DB0070B5D8
:105528000133002403A500BF5B1920C940CAAD1B85
:1055380020C0184720C940CAB54120C020C940CA68
:10554800B54120C020C940CAB54120C020C940CAC1
:10555800B54120C020C940CAB54120C020C940CAB1
:10556800B54120C020C940CAB54120C06441B4FA41
:1055780084F0400970BD00BF2DE9F04F08B4F8CAA7
:1055880004B451F8042BA3FB028940F8048B4FF0B4
:10559800000AE4FB629A4FF0000BE5FB62AB4FF0A8
:1055A800000CE6FB62BC4FF0000EE7FB62CE51F840
:1055B800042B4FF00008E3FB628940F8048BE4FBFE
:1055C800629AE5FB62ABE6FB62BCE7FB62CE51F890
:1055D800042B4FF00008E3FB628940F8048BE4FBDE
:1055E800629AE5FB62ABE6FB62BCE7FB62CE51F870
:1055F800042B4FF00008E3FB628940F8048BE4FBBE
:10560800629AE5FB62ABE6FB62BCE7FB62CE51F84F
:10561800042B4FF00008E3FB628940F8048BE4FB9D
:10562800629AE5FB62ABE6FB62BCE7FB62CE40F840
:10563800049B40F804AB40F804BB40F804CB40F8A6
:1056480004EB0CBC052B00F01E810C68A0F11400C3
:10565800A1F11401A2F1140252F804EB4FF0000575
:1056680050F8046BE4FB6E5652F804EB50F8047BD8
:10567800E4FB6E6752F804EB50F8048BE4FB6E7899
:1056880052F804EB50F8049BE4FB6E8952F804EBE3
:1056980050F804ABE4FB6E9AA0F1140052F8044BE6
:1056A80051F804EB4FF0000CE4FB6EC540F804CB56
:1056B80051F804EBE4FB6E5640F8045B51F804EB38
:1056C800E4FB6E6740F8046B51F804EBE4FB6E787A
:1056D80040F8047B51F804EBE4FB6E8940F8048B36
:1056E80051F804EBE4FB6E9AA0E80006062B00F0E4
:1056F800CA800C68A0F11800A1F11801A2F11802E3
:1057080052F804EB4FF0000550F8046BE4FB6E56BA
:1057180052F804EB50F8047BE4FB6E6752F804EB94
:1057280050F8048BE4FB6E7852F804EB50F8049BB5
:10573800E4FB6E8952F804EB50F804ABE4FB6E9A74
:1057480052F804EB50F804BBE4FB6EABA0F1180070
:1057580052F8044B51F804EB4FF0000CE4FB6EC513
:1057680040F804CB51F804EBE4FB6E5640F8045BB8
:1057780051F804EBE4FB6E6740F8046B51F804EB56
:10578800E4FB6E7840F8047B51F804EBE4FB6E8987
:1057980040F8048B51F804EBE4FB6E9A40F8049B44
:1057A80051F804EBE4FB6EABA0E8000C072B6AD0C1
:1057B80008B40C68A0F11C00A1F11C01A2F11C02A4
:1057C80052F804EB4FF0000550F8046BE4FB6E56FA
:1057D80052F804EB50F8047BE4FB6E6752F804EBD4
:1057E80050F8048BE4FB6E7852F804EB50F8049BF5
:1057F800E4FB6E8952F804EB50F804ABE4FB6E9AB4
:1058080052F804EB50F804BBE4FB6EAB52F804EB1F
:1058180050F804CBE4FB6EBCA0F11C0052F8044B1A
:1058280051F804EB4FF00003E4FB6E3540F8043BFD
:1058380051F804EBE4FB6E5640F8045B51F804EBB6
:10584800E4FB6E6740F8046B51F804EBE4FB6E78F8
:1058580040F8047B51F804EBE4FB6E8940F8048BB4
:1058680051F804EBE4FB6E9A40F8049B51F804EB02
:10587800E4FB6EAB40F804AB51F804EBE4FB6EBC00
:10588800A0E8001808BCBDE8F08F002310B51C463E
:105898005AB2914200DC10BD40F823400133F7E7CB
:1058A80010B500231A465CB2A14203DCB2FA82F0BA
:1058B800400910BD50F8234001332243F3E74A1151
:1058C800012350F8220001F01F0103FA01F10840FA
:1058D8007047013949B20A06CBB205D4013900EB49
:1058E80081025268002AF6D001335BB273B103F12A
:1058F8008042013A50F82220002022B9013B00EBF7
:10590800431318B2704752080130F6E7184670473B
:1059180010B500235CB2A24200DC10BD51F8234050
:1059280040F823400133F5E710B5013A52B21306A7
:1059380001D5002010BD50F8224051F822309C4279
:1059480005D802F1FF32F2D24FF0FF30F2E7012022
:10595800F0E700EB81010023884200D3704751F83B
:10596800042D43EA52030B60D307F5E770B59DF9A0
:1059780010401E4623460546FFF79EFD30B92246D5
:1059880029463046FFF7D0FF012807D02346324684
:1059980029462846BDE87040FFF7BEBD70BD70B50A
:1059A8009DF910401E4623460546FFF7B5FD38B160
:1059B8002346324629462846BDE87040FFF77CBD9D
:1059C80070BD2DE9F04FB5B004AD9DF9F8401F4604
:1059D800814623462846FFF7CFFD24AB21463846AB
:1059E800CDE90235FFF775FFC0EB841005B26B42B5
:1059F80003F01F034FF0200695FBF6F676B205F08C
:105A08001F0814A858BFC3F100083146FFF73DFF2F
:105A1800B8F1000F30B22DDD14AB002203EB80008B
:105A2800C8F1200C1346A34219D327B27B00019377
:105A380014AB03EB870704F1FF3834AB012603EB03
:105A48008808002D53DA34AB03EB8606224656F855
:105A5800C81C4846FFF75CFF35B0BDE8F08F57F823
:105A6800236006FA08F10A4340F8232026FA0CF2CC
:105A78000133D8E714AB2246394603EB8000FFF721
:105A880047FFD2E70FFA82FE5AF8C83C53F82EB007
:105A980034AB03EB820252F8803CABEB03031B1AD6
:105AA8009B4502D034BF012000205CF8C82C42F886
:105AB8002E300131019B4AB29A42E3DB331A5E422F
:105AC800214614A85E41FFF744FF34AB03EB84037F
:105AD800214653F8802C58F8803C384643EAC27374
:105AE800013D48F8803C2DB2FFF733FFA9E734ABFE
:105AF8000021C6F1010C084603EB860A03EB8C0C67
:105B0800D8E730B51C4691B0054693F90030684691
:105B1800FFF732FDD4F8AC3069462846984711B0F3
:105B280030BD13460A46FFF7ECBF2DE9F04793F95D
:105B3800006092B00446894610463146154698469C
:105B4800FFF7AEFE002840F091804246494602A881
:105B5800FFF7E7FF434602AA21460AA8FFF7D1FF4D
:105B680002A908464246FFF7DCFF43462A46494653
:105B78004846FFF7C6FF08F104074246294628466B
:105B8800FFF7CFFF3B462A46214620460096FFF7FF
:105B9800EDFE3B462A46294628460096FFF7E6FED4
:105BA8003B462A46214628460096FFF7F8FE43461C
:105BB8002A4621462046FFF7A4FF3B4622462146B7
:105BC80028460096FFF7D2FE3B4600962A46214615
:105BD8002046FFF7CBFE2368DB074AD533463A4613
:105BE80021462046FFF768FC314682462046FFF7EB
:105BF800B0FE06F18043013B54F8230040EACA7026
:105C080044F82300424621462846FFF78AFF3B46D0
:105C18000AAA294628460096FFF7C1FE3B460AAA6B
:105C2800294628460096FFF7BAFE0AA908463B46C9
:105C38002A460096FFF7B3FE43460AAA21462046A5
:105C4800FFF75FFF02AA3B46104621460096FFF782
:105C5800A6FE324629462046FFF75AFE4946284600
:105C6800FFF756FE02A94846FFF752FE12B0BDE8FC
:105C7800F08731462046FFF76CFEC3E72DE9F04375
:105C88008BB00446154689460AAE1C22002103A89B
:105C980004F03FFC032346F8203D95F900802A468E
:105CA800494620462F1DFFF73CFF3B46324621461A
:105CB8002046CDF80080FFF772FE2B464A46214663
:105CC8002046FFF71EFFCDF800803B4605F1840211
:105CD80021462046FFF74AFE0BB0BDE8F0830000DE
:105CE800F0B5082289B00C460646FFF711FECB6ACC
:105CF80003930B6B04934B6B05938B6B0693CB6BE6
:105D08000793002708236A4669466846CDE9017764
:105D18000097FFF7D1FB082305466A46314630460F
:105D2800FFF7CAFB236B0393636B0493A36B059381
:105D3800E36B0544CDE906376A4608236946684699
:105D4800FFF7BAFB082305446A4631463046FFF799
:105D5800B3FB236A0093636A0193A36A0293A36B5C
:105D68000693E36B0793054408236A463146304699
:105D7800CDE904770397FFF79FFB636A0093A36A53
:105D8800A26B0193E36A02930492636BE26B039341
:105D9800CDE90523236A0793054408236A4631465B
:105DA8003046FFF789FBE36A0093236B0193636B2B
:105DB8000293236A0693A36A0793054408236A4655
:105DC80031463046CDE904770397FFF7A5FB236BEF
:105DD8000093636B0193A36B0293E36B0393636A72
:105DE8000693E36A07932D1A08236A46314630461C
:105DF800CDE90477FFF790FB636B0093A36B0193E6
:105E0800E36B0293236A0393636A0493A36ACDE95D
:105E18000537236B07932D1A08236A463146304607
:105E2800FFF77AFBA36B0093E36BCDE90137636A55
:105E38000393A36A0493E36ACDE90537636B079379
:105E48002D1A08236A4631463046FFF765FB2D1A9E
:105E58000D4C0FD435B9082231462046FFF764FDB2
:105E680001280FD00823224631463046FFF754FB5D
:105E78002D1AEFE70823224631463046FFF71CFB70
:105E88002D18F7D409B0F0BDC8B30700F0B5154612
:105E980089B01C4607460E461A4629466846FFF74B
:105EA80040FE23466A4639463846FFF72AFE23460F
:105EB8002A4669466846FFF724FE23466A46314665
:105EC8003046FFF71EFE09B0F0BD2DE9F0438BB058
:105ED8001446129D15F9046B00961F4680468946A4
:105EE8002B460246214602A8FFF759FD02A9129A3D
:105EF8000846FFF716FE129B02AA41464046FFF7E6
:105F080000FE129B02AA21462046FFF7FAFD2B4607
:105F18004A46394638460096FFF741FD129A3946F7
:105F280002A8FFF7FEFD02A92B4642460846009646
:105F3800FFF735FD02A92B46224608460096FFF7D3
:105F48002EFD2B464246214620460096FFF727FDA8
:105F5800129B224649464846FFF7D3FD2B4602AA24
:105F6800414620460096FFF71AFD129B2246394605
:105F78003846FFF7C6FD2B464A463946384600964E
:105F8800FFF70DFD324602A92046FFF7C1FC0BB012
:105F9800BDE8F0832DE9F047B3F9024088461E4674
:105FA80004F11F012023073491FBF3F708234FFA6C
:105FB80087F994FBF3F4944228BF144649460546F2
:105FC800FFF763FC22464146FFF76AFAB6F902304A
:105FD800E4009C421FD9E41A05EB87010022C4F1B2
:105FE80020078D420ED324364A4629463046FFF70D
:105FF8009BFC01280FD04B4632462846BDE8F047A7
:10600800FFF78ABA51F8040D20FA04F313430B6022
:1060180000FA07F2E5E7BDE8F08770B5036813F00A
:1060280001050646144605D013460A460146FFF701
:1060380043FA054621463046FFF78BFC45B104F18B
:106048008042013A56F8223043F0004346F82230A5
:1060580070BDF0B50F46A1B006461946384615463C
:106068001C46FFF71DFC20B13046FFF70EFC21B09F
:10607800F0BD224639466846FFF74AFC294608A87B
:10608800FFF746FC10A82146FFF7FFFB012318A8DD
:106098001093FFF7FAFB224608A96846FFF744FC6D
:1060A80028B9224610A93046FFF732FCDFE7009BEB
:1060B800DA0709D421466846FFF74BFC22462946F1
:1060C80010A8FFF7AAFFE6E7089BDB0707D42146DD
:1060D80008A8FFF73EFC2246294618A8F1E7002841
:1060E80023461CDD08AA69466846FFF715FA2146CB
:1060F8006846FFF72EFC224618A910A8FFF714FCE3
:10610800002805DA10A923462A460846FFF7D4F9DD
:1061180010A9234618AA0846FFF7FEF9CEE708A9F2
:106128006A460846FFF7F8F9214608A8FFF711FC68
:10613800224610A918A8FFF7F7FB002805DA18A9C6
:1061480023462A460846FFF7B7F918A9234610AA96
:106158000846FFF7E1F9BEE700487047C4B30700F7
:106168002DE9F04FEDB01F46DDF8D8810590B8F95C
:10617800026098F9004020231F3696FBF3F676B2AA
:1061880006F1FF3924AB002543F829506CAB03EB2B
:1061980089034CA88A469346394698F9012043F862
:1061A800805C43F8605CFFF77BF998F9012054A8FC
:1061B800B918FFF775F921464CA8FFF771FB074698
:1061C800002840F02E8154A8FFF76AFB02900028AF
:1061D80040F0298108F1240332464CA9184603935C
:1061E800FFF7A2FB012840F02081324654A903980A
:1061F800FFF79AFB0128069040F017811CAD0CAF01
:106208003346039A54A92846FFF723FF029B47F811
:1062180029305A46514638464346FFF7BBFE3946B1
:106228003846039B00962A46FFF7CBFB0DF5B87955
:10623800039B00962A464CA914A8FFF7C2FB2246E6
:1062480048460599FFF764FBA30009EB030A079387
:10625800059BA100591808F1440B5046FFF758FB5D
:10626800594634A8FFF754FBA3000BEB03013CA8E5
:10627800FFF74EFB08F10403494634AA2846009468
:106288000493FFF78CFB53464A463CA934A8CDF843
:106298000080FFF71AFE2346049A29462846FFF78E
:1062A800D8FE2A46514648464346FFF7EFFD029B73
:1062B800CDE9083B059B31463846CDE90A39FFF759
:1062C80008FB3146814614A8FFF703FB8145B8BF98
:1062D80081461FFA89F909F1FF3B0FFA8BFB5946F2
:1062E8003846FFF7ECFA5946071C14A818BF0127CF
:1062F800FFF7E5FA002814BF022300231F430DF11E
:10630800200A22465AF8277024A83946FFF700FBCE
:106318000DF1B00BA300F9185846FFF7F9FA21461A
:106328002846FFF7B2FAA9F10209069B2B600FFA7B
:1063380089F90DF1900AB9F1000F23DA2346049A7E
:1063480029462846FFF785FE43462A4659465046C1
:10635800FFF79CFD324651460398FFF7E5FA0128FE
:1063680004D03346039A5046FFF7D6F8013C64B28E
:106378004CAA23064BD5029BB3FA83F040096DB0B3
:10638800BDE8F08F43462A46D8F8A47059465046CF
:10639800B84749460CA8FFF792FA4946071C14A8C3
:1063A80018BF0127FFF78BFA002814BF0223002328
:1063B8001F4308AB53F8277027B32246394634A841
:1063C800FFF7A6FA079B3CA8F918FFF7A1FA43467E
:1063D8002A463CA934A8FFF759FD049B009434AA27
:1063E800514644A8FFF7DBFA5B4652463CA934A85D
:1063F800CDF80080FFF769FD434644AA29462846A0
:10640800FFF77FFB09F1FF390FFA89F993E752F893
:1064180024105AF824304B40029919430291013C48
:10642800A7E72846ABE73846A9E70298A7E7036934
:10643800C26893429CBF80681B18013B981A70473A
:106448002DE9F843D0E902940546A9EB0408406811
:10645800904520440F46144404D904F031F8EC6008
:10646800BDE8F8834246A4EB090404F029F86868FB
:10647800224607EB0801F0E72DE9F843C568064610
:10648800894617464FF000083469B3687068A5421A
:1064980028BFE418013C621B5C1BBC4228BF3C4679
:1064A800944228BF144649462844224604F008F876
:1064B800B3682544AB4208BF00253F1BA044A14454
:1064C800F560E1D14046BDE8F883000010B5114CF5
:1064D800114AA2610223C4E90433104BE361A264A8
:1064E8004FF480530E4A0F492362E26400231022BE
:1064F800E01DA3626362E362A3656365E3652265E9
:1065080004F03AF80849204604F036F82023A3712D
:1065180010BD00BF743F002074B40700FC3F00208A
:10652800EC3F00207DB4070081B4070070B5164B1E
:10653800182400FB04451D4404FB00331646DC6A9E
:10654800012C0ED0022C18D0E4B92846FFF76FFFB3
:10655800864204D832462846FFF772FF3446204662
:1065680070BD2846FFF763FF8642344628BF0446BD
:1065780022462846FFF764FFF1E72846BDE8704049
:10658800FFF77ABF0024EAE7743F0020FFF79EBFB9
:1065980041DF7047014B01221A7070471C540020DC
:1065A8000268530910B5044618D0012B40F2FF3396
:1065B80018BF002302F01F02D340DB0704D40949A7
:1065C8004FF4F670FCF73EFD23681F2B83BF03F0E2
:1065D8001F03054823604FF0A04010BD4FF0FF3364
:1065E800E8E700BF94B107000003005008B5FCF7C6
:1065F800C1FAFCF79FF80028FBD1BFF34F8F05497C
:10660800054BCA6802F4E0621343CB60BFF34F8FB7
:1066180000BFFDE700ED00E00400FA0508B50948F1
:10662800094B0A49C01AC008000440F00400FCF7EE
:10663800E5F9074B074800221A70BDE8084002F048
:10664800DFBA00BF38A6070038A6070088B40700DD
:106658001C540020F565070008B50748074B084992
:10666800C01AC008000440F00300FCF7C7F9BDE8F1
:106678000840FFF7D3BF00BF38A6070038A60700B9
:106688009EB40700042810B5044609D802280DD87E
:1066980012D00B4B1B6893B12046BDE81040184739
:1066A800831F012BF5D8FFF7B9FFF2E705494FF42F
:1066B800701000F0F5FAECE702F096F9E9E710BD82
:1066C800205400206166070008B50648064B0749B4
:1066D800C01AC008000440F00400FCF78FF900203D
:1066E80008BD00BF38A6070038A60700B2B40700E7
:1066F800F7B5774B774C7849E41AE408240444F05A
:10670800040605463046FCF779F9744B68461D6067
:1067180019230093FFF744FF009B714A03F5E073C8
:1067280040F82320002002F081FA002840F0CA80B7
:1067380000F064FC012800F0BE80022800F0C5804B
:10674800002840F0BF804FF08043D3F8005415F480
:1067580080354CD04FF48032C3F800240546614F91
:106768003B6A012B56D0604944F00300FCF746F918
:106778005E493046FCF742F94FF4701400F092FD80
:106788005B4A20211820FCF72DFB08B1FEF7A6FD77
:106798004FF08043D3F81C2502F0F802B02A09D143
:1067A800D3F81C25D20742BFD3F81C2502F04E02AD
:1067B800C3F81C25FFF788FF002840F08380204697
:1067C8004C4900F06DFA4C4800F098FE002879D149
:1067D8004A493046FCF712F900F0AAFDFCF78AFB9B
:1067E800FBF7A8FF0028F7D1FFF7D2FEF4E7D3F8AC
:1067F800202502F0F802A82A0AD1D3F82025D007CC
:1068080006D5D3F8202502F05602C3F82025A6E7BE
:106818000125A4E74FF440535A68394B9A420FD1E7
:106828007A6B1DB997F86032012B09D035484FF4BF
:10683800805103F055F818B9334944F0020095E740
:1068480002F01AFBBA6901461DB997F8A132012B6B
:1068580005D02E4803F044F808B92D49EDE72D4935
:106868003046FCF7CBF8192301A80193FFF798FEEF
:10687800019AD0F81035D340D90701D4264978E7D2
:106888004FF08043D3F81C3513F0B10F01D02349E2
:106898006FE702F04BFAA8B9214D2870214802F0A1
:1068A800AFF92B7823B920494FF40270FCF7CAFBE3
:1068B80000F03EF801E0FFF7B1FE1C4944F001008A
:1068C800FCF79CF8032003B0F0BD4FF4A02455E773
:1068D80038A6070038A60700CCB4070020540020CB
:1068E8000C000300F46B0020E3B4070081B5070037
:1068F800FC4F0020616607008D660700F0B50700B1
:10690800DBE5B151546E002011B50700956E0020EB
:106918004CB5070074B50700A4B50700C3B5070058
:106928001C5400209D65070000B60700E4B5070069
:1069380037B5184B184C194D1949E41AE4082404C2
:1069480044F004004FF480520190FCF75BF8D5F84E
:10695800802014490198FCF755F84FF0FF33C5F82B
:106968008030C5F88031C5F88430C5F8843101F02D
:10697800F3FC20B10C4944F00100FCF73FF8FBF7A9
:10698800D9FE0028FBD14FF4805003B0BDE8304059
:1069980000F032B838A6070038A6070000E100E08A
:1069A8004EB6070084B60700AEB6070080F3088825
:1069B8000847000070B50546C1F30B00A8B9B5F546
:1069C800FE2F12D80B4E3268072A10D8130103F194
:1069D800804404F5F0340132C4F80058C4F80418AF
:1069E8000221C4F80818326070BD0720FCE70420B3
:1069F800FAE700BF2454002038B504462648C0F5FD
:106A0800FE21FFF7D7FF054668B12448244B2549E6
:106A18001B1ADB081B0443F001002A46FBF7F2FFB0
:106A28002846FEF75BFC02F027FA1F4B9B6903F62A
:106A3800FF7323F47F6323F00F0319180020FFF777
:106A4800B9FF054668B11548154B18491B1ADB08EC
:106A58001B0443F001002A46FBF7D4FF2846FEF743
:106A68003DFCEFF305820023D4E9005483F3148836
:106A780083F3108883F3118883F31388C2F3080221
:106A88001AB10B495820FCF7DDFA21462846BDE823
:106A98003840FFF78BBF00BF0020070038A607006B
:106AA80038A60700E3B60700F46B00201AB7070002
:106AB8004EB7070073B5274B064627481B1ADB0855
:106AC8001B040C463246254943F00400FBF79AFFA5
:106AD800B4F1807F39D322498F20FCF7B3FA6FF0E5
:106AE8007F41A14228BF21461E4B641AD3F80455A2
:106AF800631E942B96BF9634746074600D44347B87
:106B080025F07F4598BF963D032C03D9144977207B
:106B1800FCF798FA134E04F5A8734FF4F86046F89A
:106B28002350114B43F001039847104BA200134424
:106B380000221A601B680193019B4FF4803303FA0B
:106B480004F4C6F8044302B070BD952CC7D80449B4
:106B58009020C2E738A6070038A60700ACB70700A0
:106B6800C2B707000040024040B807004041024059
:106B78001FB518490B7853BB4FF08043A024D3F8B6
:106B88001824D2035CBF01229A60134B0022C3F879
:106B98000021D3F8000103900398C3F84021D3F8EB
:106BA800400102900298C3F84421D3F844010190AF
:106BB80001980A4880F82443102444600220C3F84E
:106BC800082501229A601A60C3F804030A7004B009
:106BD80010BD00BF2C5400200040024000E100E03E
:106BE800264B2DE9F743D3F8042152B124490A680A
:106BF80001320A600022C3F80421D3F8043100935B
:106C0800009B204D204B214C214EDFF89080DFF86F
:106C18006C90204FED1AED082D0445F004053368FB
:106C2800CBB100233360336801932246414628469E
:106C3800019BFBF7E7FE227B17494FF48033934013
:106C4800C9F8083322462846FBF7DCFE616851B1D3
:106C58002046FFF72FFF0436BE4204F11004DED1B0
:106C680003B0BDE8F083A16811B12046FFF722FF09
:106C78002368002BEFD09847EDE700BF00400240A3
:106C88002854002038A6070038A60700182B002033
:106C980040410240484102402DB807001BB8070098
:106CA800F8B5114B114E0446114837681B1ADB081A
:106CB8001B043A4643F004000D460E49FBF7A2FEBA
:106CC8003A7B4FF4803393400B4AC2F808334CB1F7
:106CD8003668FFF74DFF356021463046BDE8F8407D
:106CE800FFF7E8BEF8BD00BF38A60700382B002024
:106CF80038A607001BB807000040024070B5074BD4
:106D08001D6804460E46A860FFF732FF2E60214634
:106D18002846BDE87040FFF7CDBE00BF3C2B0020E1
:106D2800034A044B1068D3F8043503EB006070473E
:106D38002854002000400240014B01221A7070477D
:106D48002D540020224BDA6AAC2A2DE9F3415F6A00
:106D58009D6C1FD15B6B1D44FF1A1E4B1E4E1F4AB4
:106D68001F490097F61AF608360446F004082B4621
:106D78004046FBF75AFE19483A46294603F069FB94
:106D8800044668B917494046FBF738FE204602B06A
:106D9800BDE8F081002DE0D102F082F80546DCE77D
:106DA80011493B462A464046FBF735FEFBF7C2FC35
:106DB8000028FBD100F0BCFA3946284601F0AEFAAB
:106DC80004460028E2D0094946F00100DCE700BF8C
:106DD800F46B002038A6070038A60700002007003B
:106DE80046B807007BB80700B2B80700DFB807004D
:106DF8002DE9F04F3C4B16463C4A9B1A87B0DB08FE
:106E08001B04814205460F46049343F0040B08D146
:106E180037495846FBF7F2FD0024204607B0BDE885
:106E2800F08F03D233494F20FCF70CF936B1C5F384
:106E38000B031BB12F495320FCF704F97B1BB3F557
:106E4800805F4FEA133403D22A495720FCF7FAF837
:106E580000F028FA082C28BF082406F6FF79230337
:106E68004FEA1939039405930EB93446D5E7039BC5
:106E78004B453ABFDDF80CA0DDF81480CA464FF048
:106E880000025146284628BFB04601F001FA0446E0
:106E98000028C2D11849CDF800802B463A465846FA
:106EA800FBF7C3FD08F10302234622F0030239462B
:106EB800284601F0AFF904460028AED10F4A136BFB
:106EC8004344136301F0A2FEA9EB0A09A6EB0806E6
:106ED8004544474404460028C6D0049B084943F06B
:106EE8000100FBF78BFD98E738A6070038A60700D6
:106EF800F9B8070008B9070064B90700F46B002067
:106F080085B907002DE9F74301F0DAFF314C324B20
:106F1800DFF8E4903149D9F84860D9F83080D9F8D9
:106F28003450E41AE4082404074644F004000190AD
:106F3800FBF764FD06F5005301985A68284B9A42FE
:106F480009D0284944F00100FBF758FD03252846DD
:106F580003B0BDE8F083D9F83030AB421E4404D109
:106F68002149FBF74BFD0025F1E7C3B94FF4405227
:106F78001178142982BF1D495269B2FBF1F206F556
:106F8800005198BF1A4691F800C0BCF1140F82BF97
:106F98004969164BB1FBF3F31549FBF73CFDA5EB2B
:106FA800080202F6FF7222F47F6222F00F023146D5
:106FB80007EB0800FFF71CFF054628B10D4944F010
:106FC8000100FBF71BFDC2E703B0BDE8F04301F089
:106FD8001DBE00BF38A6070038A60700BEB90700C7
:106FE800DBE5B151E3B9070017BA070040420F00CB
:106FF80029BA070052BA0700F46B00202DE9F047C0
:10700800624B634D634E6449ED1AED082D0445F05B
:1070180004073846FBF7F2FCF36AAA2B00F09A80C3
:107028000CD8012B22D0A52B00F0888045F0030056
:107038005A49FBF7E3FC0020BDE8F087AC2BF5D1FB
:1070480057493846FBF7DAFC56493846FBF7D6FC71
:10705800FFF758FF0446002800F08680524945F0A3
:107068000100FBF7CBFC4FF0010823E04F493846FD
:10707800FBF7C4FCD6F82490D6F848A001F0FCFE33
:10708800346B4B4900EB04083846FBF7B7FC316B0F
:107098005144884514BFA9EB040200224046FFF77B
:1070A800A7FE044670B1434945F00100FBF7A6FC72
:1070B8004FF00008F36A4049224645F00100FBF70B
:1070C800AAFC13E001F0D8FE22464946FBF79EFFD2
:1070D800B26A904280462AD138493846FBF78EFC7E
:1070E8000123C6E90783C6F81890A0463448DFF89C
:1070F800F49001F0B7FE0023324889F8003001F01F
:1071080085FD99F80030044623B92F4940F2A510AF
:10711800FBF798FF8CBBB8F1000F35D0336A012B11
:1071280032D138462949FBF769FC022084E7034637
:10713800274945F00100FBF76EFCD6E7254938469C
:10714800FBF75CFCFFF7DEFE4FF001080446002C5D
:10715800CCD0AFE720493846FBF750FCFFF7F2FDEB
:107168004FF000080446F2E7FFF7ECFD044608B1CB
:107178001A4974E74FF00108B8E745F001001849CB
:10718800FBF73CFC032057E7012055E738A607002A
:1071980038A60700F46B00206BBA070077BB07001E
:1071A80020BB07002EBB07004BBB07008CBA0700AB
:1071B80096BA070052BA070090BB0700B1BA070099
:1071C800186C0020416D070008B90700C2BB070012
:1071D800C6BA07000EBB070017BB070061BB070054
:1071E8001EBC07002D54002010B50024D4F8F83F29
:1071F800013304D1084940F6F870FDF7B3F8D4F824
:10720800FC3F013307D1BDE810404FF4FC2140F6A4
:10721800FC70FDF7A7B810BD002007000A4AD2F895
:1072280000347BB109480023D2F80815D940C907B2
:1072380048BF03F5C07103F1010348BF42F82100BC
:10724800072BF1D1704700BF000001403546526E50
:1072580008B50748074B0849C01AC008000440F0A1
:107268000300FBF7CBFBBDE80840FFF7D7BF00BF23
:1072780048A6070038A6070038BC070007B5084B22
:107288000022C3F80021D3F800310193019BFBF7DA
:1072980071FCFBF74FFA0028FBD103B05DF804FB43
:1072A8000000014037B5194D2B784BBB18481949D8
:1072B800194B401AC008D3F80024000440F003001A
:1072C80002B3D3F80445154901902246FBF79AFB0F
:1072D80040F616529442B8BF1446A4F54864FFF726
:1072E8009DFF01980E492246FBF78CFB0D4920466D
:1072F800FFF704FD0C4B4FF480321A6001232B700A
:1073080003B030BD0949FBF779FBF7E72E5400209D
:1073180048A6070038A607000000014046BC070041
:107328005FBC07005972070000E100E091BC07004C
:10733800034BD3F800340BB1FFF770BF704700BFA1
:10734800000001404FF08053D3F830210D2A55D169
:107358004FF080410022C1F80C21C1F81021C1F87A
:1073680038254A4AD3F80404C2F82005D3F808049B
:10737800C2F82405D3F80C04C2F82805D3F8100481
:10738800C2F82C05D3F81404C2F83005D3F8180451
:10739800C2F83405D3F81C04C2F84005D3F8200419
:1073A800C2F84405D3F82404C2F84805D3F82804E1
:1073B800C2F84C05D3F82C04C2F85005D3F83004B1
:1073C800C2F85405D3F83404C2F86005D3F8380479
:1073D800C2F86405D3F83C04C2F86805D3F8400441
:1073E800C2F86C05D3F84434C2F87035D1F80034CB
:1073F800DB0744BF6FF00103C1F80034244AD2F818
:10740800883043F47003C2F88830BFF34F8FBFF35E
:107418006F8F4FF01023D3F80022002A03DBD3F834
:107428000432002B2EDA1B4B0122C3F80425D3F8B3
:107438000024002AFBD04FF010221221C2F80012BB
:10744800D3F80024002AFBD04FF010231222C3F8EF
:107458000422104BD3F80024002AFBD00022C3F8E2
:107468000425D3F80024002AFBD0BFF34F8F084926
:10747800094BCA6802F4E0621343CB60BFF34F8F35
:1074880000BFFDE7054B064A1A60704700C0004080
:1074980000ED00E000E001400400FA05402B002068
:1074A8000090D00313681F2B10B5144607D900228B
:1074B8000830FCF7B8FE08B92023236010BD48F255
:1074C8001450FBE70830FCF78BBE0830FCF758BEB9
:1074D800008800F001007047831F012B10B5044697
:1074E80002D8002001F084FC034B1B681BB1204626
:1074F800BDE81040184710BD3054002038B5104B77
:10750800104C1860104B1149E41AE408240444F0A4
:107518000300FBF773FA0020FFF7DEFF0C4801F0C9
:107528002DFC054620B9BDE83840094801F0D2B91C
:107538000246084944F00100FBF764FA284638BDC2
:107548003054002038A6070038A6070084BE07007C
:10755800E174070097BE07006CDF70476DDF704766
:1075680072DF704773DF704774DF704775DF7047ED
:1075780076DF70477ADF70477CDF70477DDF7047C2
:107588007FDF704786DF70478FDF704790DF704777
:10759800A8DF7047AADF7047ADDF7047AEDF7047DE
:1075A800B0DF7047B1DF7047B5DF704762DF704703
:1075B80066DF704713DF704710B5094B0949044669
:1075C80009481B1ADB081B04224643F00400FBF79A
:1075D80019FA21460548BDE81040FBF7B3BE00BFC5
:1075E80050A60700C1BE070038A60700BCA60700C2
:1075F80070B518228CB00DEB0200002102F089FF53
:10760800282308932348244B2449254CC01AC00832
:107618000004012540F004008DF818508DF82D5015
:10762800FBF7ECF91623ADF806300023CDE9033358
:107638000593022306222370237159230926A27079
:1076480063710322FE236570E270A3710DF10601D8
:10765800A0190294ADF80C60FFF790FFB8B9BDF817
:10766800063026725A19E271BDF80C200D4C1344ED
:1076780002A906AA2046ADF80C30FFF771FF30B911
:107688002078FFF771FF20782946FFF76BFF0CB0D1
:1076980070BD00BF50A6070038A60700D3BE07007C
:1076A800B2640020442B0020F0B50388242B8FB04F
:1076B800044651D80BB90FB0F0BD013B232BFAD8C3
:1076C80001A252F823F000BFC17A0700BF76070075
:1076D800BF760700BF760700BF760700BF760700B2
:1076E800BF760700BF760700BF760700BF760700A2
:1076F800BF760700BF760700BF760700BF76070092
:10770800BF76070091770700D577070079790700DA
:107718002D790700CD7B0700BF760700BF760700ED
:10772800BF760700BF760700BF760700EF7B07002C
:10773800BF760700BF760700BF760700BF76070051
:10774800B5790700BF760700137A0700F5790700B7
:10775800E17807000F790700503B9AB2062AAAD8A9
:10776800062BA8D801A252F823F000BF037807001F
:10777800CD7A0700EF7B0700BF760700BF760700CA
:10778800897807003B7A0700AF4BB04DB049B14E3E
:10779800ED1AED082D0445F00400FBF72FF9A38836
:1077A8003380AD4B1B680BB101209847AB4930883B
:1077B800FFF7DCFE024600283FF47DAFA84945F0FC
:1077C80001000FB0BDE8F040FBF71CB9A14B4FF624
:1077D800FF721A80A34B1B685A0704D4FFF708FFEF
:1077E80008B1FDF77BFD9C4B1B68002B3FF463AF92
:1077F80002200FB0BDE8F04018479B4FE288BB88D5
:107808009A427FF458AF9948904DFBF76FFD8E4B25
:10781800ED1AED082D04064638B9954945F00200E1
:107828000FB0BDE8F040FBF7E9B8F4230093238AD2
:107838009049024645F00400FBF7F7F8228A04F164
:107848001201304602F03CFE1822002108A802F07E
:1078580060FE08238DF82030874B0A93874B0997E1
:10786800CDE90B3608A8238AADF8343001F012F8B8
:1078780000283FF420AF7D483146FBF763FD1AE747
:10788800E288F62A24D8D31E9B0723D0D31F9BB2A5
:10789800013B594201F0030103F0030302F1FF34F5
:1078A80058BF4B42E31A9CB2674B68487449C01AE8
:1078B800C0080004234640F00400FBF7ACF8654B11
:1078C80021461888FFF770FE00283FF4F4AE88E0E0
:1078D800F724E9E71446E7E75B4B5C486949C01AB7
:1078E800C008000440F00400FBF788F80022A088D4
:1078F80008A9CDE90822FFF749FE00283FF4DBAECE
:10790800FDF7ECFCD7E6504B504862895E49C01A37
:10791800C008E389000440F004000FB0BDE8F0405F
:10792800FBF779B8484B494C58494A4DE41AE408E2
:10793800240444F004042046FBF760F8022308936B
:10794800288806AB08AA42F605210993FFF724FE0A
:1079580008B1FDF7C3FCBDF818204D492046FBF7D8
:1079680051F8002328881A468521FFF709FEC4E745
:10797800354B36484749C01AC008000440F0040097
:107988000390FBF73BF8628943490398FBF73AF801
:10799800228942490398FBF735F8A28940490398A0
:1079A800FBF730F8E2893F4903980AE7264B274D51
:1079B8003D49ED1AED082D0445F00400FBF71EF8CB
:1079C800244B04F108011888FFF7D0FD044600286D
:1079D8003FF471AE0246354945F00100FBF712F855
:1079E80020460FB0BDE8F040FDF778BC164B1748AD
:1079F8002F49C01AC008237A00930004637AA27A38
:107A080040F00400FBF711F855E60F4B0F482949E1
:107A1800C01AC008000440F00400FAF7EFFF002382
:107A2800A0888DF8203008A98DF82130FFF7ACFD2B
:107A380063E7A379002B7FF43EAE064B1321188829
:107A4800FFF796FD40E700BF38A6070050A60700DD
:107A5800E2BE0700462B0020D864002016C40700A9
:107A6800ECBE0700D46400209E640020BCA607007A
:107A78001ABF070039BF0700317D0700C17507002D
:107A880059BF07009FBF0700D0BF07000EC00700FF
:107A980036C0070059C0070080C0070096C007001D
:107AA800ACC00700BEC00700D3C0070002C1070072
:107AB80037C1070071C10700544B00211888FFF730
:107AC80077FD01E7A379002B3FF4F5AD022B7FF496
:107AD800F2AD4F4D2189AA8991427FF4ECADA27B8A
:107AE800012A7FF4E8AD4FF480320992228A474E8A
:107AF800ADF82820628AADF82A2004F114020B920E
:107B080005AF298A3088089306AA06930797FFF7D6
:107B180043FD60B93846FFF7DBFC40B940F2FD137E
:107B28003088ADF8243008A9FFF73AFDC3E50023F3
:107B380008A93088ADF82430FFF732FD0146002847
:107B48007FF4B9AD182208A802F0E3FC237D314A7E
:107B58008DF82030022B09950A9222D0062B0ED0E0
:107B6800012B0ED12C4801F043F92C4B1A882C4BD1
:107B78001A80637D0C93D4F816300D9301E0637D71
:107B88000C9308A800F086FE00283FF494AD254A1F
:107B9800254B26499B1ADB081B04024643F00100CB
:107BA8000FE6204B20482249C01AC008000440F0C4
:107BB8000400FAF723FF194AB4F815301380184A5D
:107BC8001380DEE7174B18481A49C01AC00800048A
:107BD80040F00400FAF712FF0023A0881A4619465D
:107BE800FFF7D0FC70E60023A0881A461946FFF775
:107BF800D9FC08B1FDF772FB0B480A4B0E49C01AB5
:107C0800C008000440F004000AE600BF462B00202C
:107C18009E640020317D070024A60700DC64002054
:107C2800DE64002038A6070050A60700ACC1070094
:107C38009AC10700E0C1070006C2070070B5204ED0
:107C4800346814F0010432D01E4B984236D01E4BD3
:107C58001E4D1F4C1F49ED1AED082D0445F0040573
:107C68002846FAF7CBFE22884FF6FF739A4220D0B7
:107C780019492846FAF7C2FE3368208843F00403FE
:107C880013213360FFF774FC044680B9134EC824EF
:107C980046F001064FF47A40B047013CFAD102F0B1
:107CA800AFF9044618B90E492846FAF7A7FE204648
:107CB80070BD0C4B1878FFF757FCF0E70024F6E787
:107CC800D464002024A6070038A6070050A60700A1
:107CD800462B002028C2070045C2070010C4070031
:107CE80054C20700442B00207FB50023CDF80B3089
:107CF8008DF80F300A4BADF806109B89ADF80830A7
:107D080001238DF80A300DF10603CDE90430054B47
:107D180002A91888FFF742FC07B05DF804FB00BF12
:107D28009E640020462B002030B50D4687B00446DF
:107D380020B9464940F29110FBF784F925B9434927
:107D48004FF4C970FBF77EF900210D2202A80191BA
:107D580002F0DFFB2378082B0BD13D4A3D491388FD
:107D68000988013B9BB2138031B32BBB03231180DD
:107D78002370637822788DF805206021012B8DF817
:107D880004108DF8063019D033493448401AC00819
:107D98000004334940F00200FAF73DFE63780B2BEC
:107DA80012D100F0B1FA8DF80700002000F0A6FA11
:107DB800042101A8FFF798FF07B030BD062A05D0B7
:107DC800082A29D0032A27D00321F2E7E1688DF891
:107DD8000710D4E90123080A8DF80800080C090ED9
:107DE8008DF80A10110A8DF80B208DF80C10110C63
:107DF800120E8DF80E201A0A8DF80F308DF810200B
:107E08001A0C1B0E8DF80D108DF809008DF8112035
:107E18008DF812300F21CCE7D4E90123110A8DF82F
:107E280007208DF80810110C120E8DF80A201A0A76
:107E38008DF80B308DF80C201A0C1B0E8DF80910DC
:107E48008DF80D208DF80E300B21B2E76DC20700BA
:107E5800DE640020DC64002038A6070050A6070076
:107E6800C0C207002DE9F041054694B020B9404949
:107E780040F26240FBF7E6F83E4B4FF6FF721A807D
:107E880001204FF659632A4602A98DF80A00ADF879
:107E98000830FFF77DFB0446002865D1364B04AA5D
:107EA80003F11007164618685968144603C40833C6
:107EB800BB422246F7D1A91C3046FFF777FB0446A0
:107EC800002851D101461C220DA802F022FB9DF882
:107ED80034308DF8044043F004038DF83430022325
:107EE800ADF80C30AB788DF80E3003238DF80630E2
:107EF800F423CDE90A44ADF82C302B464FF0110895
:107F080033F8040B0C9403AF01AE08AA0DA98DF841
:107F1800058008970996FFF73DFB044620BB0146FC
:107F28001C220DA802F0F5FA18238DF8343001232D
:107F3800ADF80C30AB788DF80E3013238DF8063081
:107F48001723CDE90A44ADF82C302B4608AA33F89C
:107F58000C0B8DF804400DA90C94CDE908768DF82A
:107F68000580FFF717FB0446204614B0BDE8F081F2
:107F78006DC20700462B0020F8C307002DE9F04327
:107F88005A4E87B0336813F0010400AF804640F0C2
:107F9800AA80574B574D5849ED1AED082D0445F066
:107FA80004052846FAF72AFD544B5548C3F80080C3
:107FB800FBF75EF97C6000F0C2F90446002873D133
:107FC800504A51492846FAF71DFD4E48FFF7F2FA84
:107FD8000446002868D14D492846FAF70FFD01F0FC
:107FE800D1FF044600285FD1381D02F09DF80446F1
:107FF800002859D146492846FAF700FD391D0120C5
:1080080002F09CF8044600284ED142492846FAF767
:10801800F5FC381D02F052F90446002844D100F05E
:1080280075FE002845D03C4800F060FE336843F0F8
:10803800020333604FF01108381D87F80080FFF7FE
:108048008DFAE946044678BB7B79381D01337B718C
:10805800FFF782FA0446A0B933689B072ED52E4C49
:108068002E49A369221D2846FAF7D5FC228B211D2B
:108078003846FFF781FA044618B92948FFF77AFA13
:108088000446CD4684B92748FFF7ECFE044658B9A4
:10809800FFF7AEFA044638B93368234943F00103C1
:1080A80028463360FAF7AAFC20461C37BD46BDE8CF
:1080B800F0831E492846FAF7A1FCBBE71C4928466D
:1080C800FAF79CFC1B4A516810681B4A3B1D03C306
:1080D8002D233B731368C7F80D305368C7F8113068
:1080E8004246391DC4E70024DEE700BFD4640020FF
:1080F80038A6070050A60700E7C20700D86400208A
:10810800BCA607000020070006C3070026C3070017
:108118003BC3070052C307003454002084C3070040
:1081280016C407009E640020CDC307006AC3070079
:10813800A5C30700C4C307005D3F002030B51A4936
:108148000B6885B004460BB1013B0B601748184A11
:1081580063682578121AD208120442F004008BB919
:108168000B68144A14490093012D08BF0A46A368F6
:108178001249FAF75AFC63699BB1E06805B0BDE89B
:10818800304018470A68029222690192A2680A4997
:108198000092084A012D08BF0A460949FAF75FFC10
:1081A800E9E705B030BD00BFE064002038A607004D
:1081B80058A6070024C407001EC407002AC40700E5
:1081C80050C4070008B502460B4B0C481B1ADB08C5
:1081D8001B0443F004004AB10949FAF70FFC0949A6
:1081E8000948BDE808400022FBF7EABA0749FAF750
:1081F80005FC0749F4E700BF58A6070038A60700A2
:108208008CC40700A8AA0700FC2A0020B2C40700F3
:108218007CAA07002DE9F7439846174C174BDFF85F
:108228006C90E41AE408D9F800302404CDE900235E
:1082380005460B460E4617461149024644F004000F
:10824800FAF7FFFB29460F48CDF800803B46324637
:10825800FBF708FB054640B9D9F800300133C9F8E7
:108268000030284603B0BDE8F0830246064944F0D2
:108278000200FAF7C7FBF4E758A6070038A607007C
:10828800DAC40700FC2A00201DC50700E0640020AE
:108298002DE9F341134B144C144FE41AE4083B68DE
:1082A8000093240405460B460E46904610490246A4
:1082B80044F00400FAF7B9FB29460E484346324613
:1082C800FBF720FB054630B93B6801333B60284685
:1082D80002B0BDE8F0810246074944F00200FAF70F
:1082E80091FBF4E738A6070058A60700E0640020D1
:1082F8004AC50700FC2A002087C50700014B1870F3
:108308000B207047E4640020024B002218781A7092
:10831800704700BFE464002018DF704730B585B0AF
:10832800054610220C466846002102F0F2F8A4081F
:10833800684601950294FFF7EFFF05B030BD1FB501
:108348000023CDE901330393684602230093FFF726
:10835800E3FF05B05DF804FB4FF000534FF4805283
:108368001A60002070470000084B09480949C01AE4
:1083780010B5C008000440F00400FAF73FFB064BB4
:10838800BDE810401B680620184700BF38A6070044
:1083980060A60700C2C50700F06400200A2803D9B8
:1083A8000B38C0B2FFF7AABF7047000070B505468A
:1083B80086B00020FBF7E2FA0146A0B1274A18214F
:1083C8002846FAF733FD00283DD0254A254B264993
:1083D8009B1ADB081B04024643F0010006B0BDE807
:1083E8007040FAF70FBB1822684602F092F804238F
:1083F8001C4C8DF800301A4B1C4EE41A1C4B1A6D9D
:108408003368E40824049A4244F004041DD119494D
:108418002046FAF7F3FA184B3168186801F06AFC3D
:108428008DF80100FFF7BAFFD5E901138DF80100B7
:1084380068469847114800F0E9FB9DF8012010496B
:108448002046FAF7DFFA06B070BD01238DF8013037
:108458006846D5E901139847EFE700BFB5830700E1
:1084680038A6070060A60700F6C50700E8640020E4
:10847800F46B00201FC60700EC640020718307001E
:108488004EC607002DE9F041836888B0044623B939
:10849800974940F2CF20FAF7D5FD1822002102A80B
:1084A80002F037F80123934E8DF80930924B227869
:1084B8008DF80820F61AF6083604531E46F004050F
:1084C8000B2B00F2C581DFE813F02C000C002C0008
:1084D8002C00C3012C00C3012C00C301C301C3013C
:1084E800110086492846FAF789FA07E028468449A0
:1084F800FAF784FA834B07201B6898479DF80920F0
:1085080081492846FAF77EFAD4E9011302A8984768
:108518009DF80930012B00F085817A4B05201B68F6
:108528007FE1062A794F01D0012A01D122693A70E8
:108538003A78012A09D0022A74D0754946F0010018
:10854800FAF75CFA00233B70C6E0072B64D8DFE833
:1085580003F004631443635B631E6E492846FAF70D
:108568004DFA684B03201B689847606901F092F840
:10857800FFF714FF8DF80900C0E767492846FAF7A6
:108588003DFA664BDA6B1B6C03920493B6E72369DA
:1085980023B9574940F21310FAF754FDA38A23B9B7
:1085A80053494FF48A70FAF74DFD5D492846FAF7AA
:1085B80025FAA18A206901F085F8FFF7EFFE574BED
:1085C8008DF80900DA6B1B6C0493E3680392002BA7
:1085D80094D02069984791E752492846FAF70EFA4D
:1085E8005149524801F0ECF8FFF7D8FE01288DF800
:1085F800090083D1002000F009FB08B94C4971E754
:108608000A238DF8093079E74A492846FAF7F6F936
:108618004FF400730593B4E735494FF4BC70FAF78B
:1086280011FD6BE7072B00F20F81DFE813F008005C
:108638000D01CF00DE000D01FE000D0195003E4941
:108648002846FAF7DBF901F06DF830B93B4946F0F6
:108658000100FAF7D3F90823D3E7626932B9384938
:1086680046F00100FAF7CAF90323CAE7C2F30B037D
:1086780043B12A4B2C495B6D096813448B4201D0E6
:108688003049EDE7B2F5805F06D92F4946F0010081
:10869800FAF7B4F90423B4E7204F23497B6D09683E
:1086A800D018884206D9009146F001002749FAF708
:1086B800BCF9D0E77A64FA6CBA641C4A3B65106866
:1086C8003B63002201211844FFF7E2FD30B1204945
:1086D80046F00100FAF792F9052392E7BB6C009384
:1086E8003B6D7A6C1B492846FAF79FF906E700BFED
:1086F80076C6070060A6070038A60700CDC60700A3
:10870800F1C60700F06400204EC60700482B002081
:1087180089CA070009C7070033C70700F46B0020A0
:1087280057C7070080C70700E8640020EC640020F2
:10873800ABC70700D0C70700FAC7070021C8070062
:1087480056C807006FC8070090C80700B4C80700DC
:1087580025C907003CC9070041492846FAF74EF9E0
:1087680000F0E0FF00283FF476AF3E4FA18AD7E93A
:1087780014329B1A7A6C0B44934201D93A496FE739
:108788003A4A3B6B1268206903EB020807F148027A
:10879800FAF73CFCE368064623B935494FF4F8700C
:1087A800FAF750FCE368A28A21694046FFF732FDD8
:1087B80008B1E3680DE7A38A3A6BBE641A443A63CA
:1087C8003A6D049613443B65039397E6254E294971
:1087D8002846FAF713F9B36C326D27492846FAF799
:1087E8001AF9B36C0493336DEEE728462349FAF778
:1087F80005F91C48D0E91473426CFB1A934205D062
:108808001F4946F00100FAF706F924E7836CC364B0
:108818000021416447652046FFF7C8FD194B1B68D6
:108828000420984708B0BDE8F08117492846FAF7B0
:10883800E5F80C4B4FF480519A6C1B6D0591009133
:108848000492124903934EE7094940F29720E6E65D
:108858000F4946F00300FAF7D5F80223D1E600BF26
:1088680077C90700F46B00209DC90700EC6400205D
:1088780076C60700B4C90700D5C90700EBC90700C9
:1088880013CA0700F064002037CA07005ECA070051
:10889800A9CA0700836810B58BB10A4A1821FAF7EC
:1088A800C5FA044648B10848084B09491B1ADB08B1
:1088B8001B0443F00200FAF7A1F8204610BD072474
:1088C800FBE700BF8D84070038A6070060A60700F5
:1088D800C8CA070038B50546C0B10120FFF772FCC9
:1088E800044648B900F0C8FE00F01CFF30B9084B38
:1088F80000201D60FFF702FD204638BD05490648E7
:1089080000F05EFF0128F2D00324F5E70724F3E71F
:10891800F0640020E8640020EC6400202DE9F743AF
:1089280017464FF4607298461F4D0646894601F077
:1089380090FD1E4BED1AED0804462D0445F0040089
:1089480054B91B49FAF75AF81FB9002003B0BDE81B
:10895800F0832046B847F8E716490190FAF74EF831
:10896800154901983246FAF74DF8002201213046A0
:10897800FFF78EFC30B1114945F00100FAF73EF8D7
:108988000320E3E74FF460724946404601F098FD42
:108998003B464FF4607241463046FFF73BFC0028E7
:1089A800D3D00749E8E700BF68A6070038A6070044
:1089B800F8CA070042CB070056CB070076CB070062
:1089C80099CB07000368013310B5044609D000228B
:1089D80058210430FAF71AFB23681B1A58425841E9
:1089E80010BD0020FCE700002DE9F0474C48DFF8F7
:1089F8005C814C4CDFF858914B4EFFF7E3FFD8F8F9
:108A080000A007465046FFF7DDFF0546002871D055
:108A1800DAF80450012D0AD00022C3210AF5187093
:108A2800FAF7F4FADAF85C522B1A5D425D41002F2E
:108A380050D0A4EB0907FF083F0447F004073B495F
:108A48003846F9F7DBFF364937484FF4607201F0D2
:108A580037FD8DB136493846F9F7D0FFD8F80050C0
:108A680034485422291D01F02BFD33484FF432724B
:108A780005F15C0101F024FD7768012F4DD1A4EBCD
:108A88000900C0082D4C2E49000440F00300A4F54D
:108A9800E475F9F7B3FF0FCD0FC40FCD0FC40FCD99
:108AA8000FC495E80F0084E80F0004F11005A4F541
:108AB800DC740FCC0FC594E80700002386F86032F9
:108AC80086F8E232F36986F8A17285E80700C6F8ED
:108AD800A23220E085B1A4EB0900C00800041949BE
:108AE80040F00300F9F78AFFD8F800100E484FF459
:108AF8006072BFE7002F9CD1A4EB0900C0080004F6
:108B0800114940F00200F9F779FF07484FF4607205
:108B1800002101F0FEFC02237360BDE8F08700BF6E
:108B280000F0070068A60700F46B0020C0CB070020
:108B3800D5CB0700F86B0020506C0020186F002080
:108B4800BCCC0700FFCB070058CC07004C2B0020FB
:108B580038A6070070B50C4C054600225821201D88
:108B6800FAF754FA00222060C32104F51870FAF7C6
:108B78004DFA2A46C4F85C022146044B0448BDE875
:108B88007040FFF7CBBE00BFF46B00207468002074
:108B980000F00700F8B5134B134C144FE41AE4081F
:108BA80024040D463A681249064644F00300F9F7D2
:108BB80029FF2846FFF706FF20B90E494FF4C17078
:108BC800FAF740FA32460C4B38682946FFF7A6FEFA
:108BD800024630B144F001000849BDE8F840F9F711
:108BE80011BFF8BD38A6070068A607004C2B002067
:108BF800E8CC070012CD0700F464002066CD07001A
:108C08000149FFF7C7BF00BF00F0070038B50546A8
:108C18000020FFF79FFF044618B903492846FFF7CD
:108C2800B9FF204638BD00BFF46B002037B5114BA3
:108C3800114C1249E41AE4082404054644F00400DF
:108C4800F9F7DCFE2846FFF7BDFA40B10C490246A9
:108C580044F00100F9F7D6FE032003B030BD0190BF
:108C6800FFF7C2FE0198FFF7D1FF0028F5D00549AC
:108C78000246EDE738A6070068A60700A3CD07005F
:108C8800C6CD0700F1CD070010B5084C4FF40072AF
:108C9800FF2104F15C0001F03CFC2022002104F1DA
:108CA800380001F036FC0023236310BDF46B00206C
:108CB80029DF704738B50C4D0446D5F8643378B1D0
:108CC80001330FD1002218210430FAF79FF9214609
:108CD8002060072205F55970BDE83840FFF7E8BF66
:108CE8000E2038BD0820FCE700F0070050B1064B05
:108CF80003F11C0253F8041B40F8041B9342F9D1FA
:108D0800002070470E20704764F3070010B5064C2A
:108D1800002218212046FAF779F954F8043C1B1A66
:108D28005842584110BD00BF68F3070010B50F4CFA
:108D3800D4F82433D4F864231340013313D00C4BF4
:108D48000C480D49C01AC008000440F00400F9F7A7
:108D580055FE4FF4FE20FBF7EDFAC92221464FF4E9
:108D6800FE20FBF715FB002010BD00BFF46B0020B0
:108D780038A6070070A607003CCE07002DE9F84387
:108D8800154B164CDFF86480154E1649E41AE408B2
:108D9800A6EB08062404F60844F004040746324605
:108DA8002046F9F72FFE4FF00009B14501D1002503
:108DB8000BE058F8393038469847054640B1034625
:108DC80009494A462046F9F726FE2846BDE8F883B1
:108DD80009F10109E9E700BF38A6070038A607002E
:108DE8002CA6070079CE07009DCE070024A6070011
:108DF8002DE9F843154B164C164D174F1749E41A31
:108E0800E4087F1B2404FF0844F0040406463A469D
:108E18002046F9F7F7FD4FF0000805F10409B845B9
:108E280001D100250BE059F83830304698470546FF
:108E380040B103460A4942462046F9F7ECFD284668
:108E4800BDE8F88308F10108E9E700BF38A6070084
:108E580038A6070024A607002CA60700C9CE0700DD
:108E6800EECE0700034A0023036043608360136368
:108E7800704700BFF46B00204FF44053074A59680D
:108E8800914201BF986800F6FF7020F47F6020F0DF
:108E98000F0018BF4FF48050704700BFDBE5B15199
:108EA80008B5FFF7E9FF054B9B69184400F6FF700A
:108EB80020F47F6020F00F0008BD00BFF46B002095
:108EC8004FF48050704700002DE9F04F89B00646F6
:108ED80003920793694A6A4B06919B1ADB081B04A5
:108EE80043F00404674904932046F9F787FD66496F
:108EF800DFF8E081DFF8E091DFF8E0A132462046B4
:108F0800F9F780FD069B6149002B0CBF42464A4693
:108F18002046F9F777FD039B5D49002B0CBF4246BD
:108F28004A462046F9F76EFD079B5A49002B0CBFAD
:108F380042464A462046F9F765FD4FF440535649E4
:108F48005A68564B20469A4214BF42464A46F9F799
:108F580059FD53492046F9F751FDDAF81830DAF887
:108F6800202050492046F9F756FDDAF82430DAF87F
:108F78002C204D492046F9F74EFD4FF0000B5FFAC3
:108F88008BF3BBF1010F02934CD0022B59D0FFF7A2
:108F980087FF039B0546002B42D0DAF82020531E9A
:108FA8005A425A410192414FAF4203D24049B1203F
:108FB800FAF748F8069B3F497F1BB74238BF0123A1
:108FC8005A4620460593F9F71DFD3B492A46204697
:108FD800F9F718FD3949B7422CBF42464A462046A0
:108FE800F9F710FD019B3649002B0CBF42464A4653
:108FF8002046F9F707FD059B3249002B0CBF424676
:109008004A462046F9F7FEFC059BFBB1019BEBB9EC
:109018000BF1010BBBF1030FB1D1B74224D217E01A
:10902800039ABFE7FFF728FF079B05463BB94FF4B4
:1090380040521A4B5268D21A18BF0122B2E75A4658
:10904800B0E7012301934FF48055ACE7B74209D24A
:10905800049B1D4943F00200F9F7D0FC042009B035
:10906800BDE8F08F029B33B120461849F9F7C6FCDA
:109078001748FFF7F7FE0020F1E700BF38A6070002
:1090880038A6070018CF070036CF070056CF0700CD
:1090980067CF070075CF07008ACF0700DBE5B1511E
:1090A8009ACF0700A9CF0700C9CF07000000070023
:1090B800E9CF07003AD0070044D0070059D007008D
:1090C8006ED0070081D0070092D00700BED00700FD
:1090D8000C6C002050CF07004BCF0700F46B00202A
:1090E8002DE9F04F4049414E8A6B414DDFF82891F8
:1090F800DFF828A1DFF828B185B06F465C31384623
:10910800FBF724FB97E80F004FF0000886E80F00F4
:10911800384BF3604FF447724146284689F800807F
:10912800CAF80080CBF8008001F0F3F932492A46EA
:109138003046FBF7A8FD044650B93048304B31495A
:10914800C01AC008000440F00100F9F757FC14E009
:1091580099F80090B9F1000F04D095F86C312C788B
:10916800A3B374B1264B25482749C01AC008000488
:1091780040F00100F9F742FC0024204605B0BDE8A4
:10918800F08F95F87241002CF7D0DBF80020DAF860
:1091980000103846FBF7DAFA97E80F0086E80F0068
:1091A8004FF4B272414605F5BA7001F0B2F91749A9
:1091B80005F5BA723046FBF766FD044680B90F48DC
:1091C8000F4B1349C01AC0080004BCE7002CD4D0C8
:1091D800AC79002CD1D008350E4B4C461D60CCE73D
:1091E80005F5BA75F8E700BFF46B0020C0720020DF
:1091F800A46F0020B992070014BE070078A60700E4
:1092080038A60700D0D00700FDD0070060BD0700D2
:109218001CD107007C730020A06F00209C6F0020E9
:10922800986F002010B590F8553013F0FB0F08D157
:1092380090F864202AB1846E74B30C60012420462F
:1092480010BD13F0010403D090F8564004B1846DAA
:109258009B07F1D590F85C30002BEDD00F4B026ED8
:10926800C3F5FC239A4201D81444E5E70C490D489C
:10927800401AC00800040C4940F00100F9F7CBFB84
:109288000424074B07480949C01AC008000440F0E5
:109298000100F9F7B3FBD2E70F24F2E7002007003B
:1092A80038A6070078A6070058D1070075D107002F
:1092B8005B68DA68134B9A4230B408D1124D2B68B8
:1092C80013B9124C236823B1114B00221A7030BC19
:1092D8007047D0E90131194413F9010B0028A1EBBB
:1092E8000302F9DB2B600A4B0A482260012119703E
:1092F800094B0A49C01AC008000430BC40F00400F9
:10930800F9F780BB60BD07009C6F0020986F0020B4
:10931800A06F002078A6070038A60700A6D107008E
:1093280000B591B0FBF714FF18B10D49DB20F9F730
:1093380089FE0C4920226846FBF75AFF0A490B4868
:1093480040236A46FBF75CFE18B10549E520F9F7AA
:1093580079FE074B01221A7011B05DF804FB00BFBB
:10936800C3D107004CB20700D072002064B10700D7
:10937800746F00202DE9F047A4B081460E461746C9
:10938800984678222023002106A80493DDF8B0A08F
:1093980001F0BFF800230593424B1B780BB9FFF788
:1093A800BFFF4148414C4249241AE408240444F0D0
:1093B80003052846F9F722FB46B944F002003D4967
:1093C800F9F71CFB132024B0BDE8F087B9F1000FB2
:1093D80005D028463849F9F711FB1620F3E7374935
:1093E80052462846F9F70EFB04AB0193344B009321
:1093F80034495346424606A8FBF790FE00284ED152
:10940800402F4CD1304B314606F140021F4651F8EF
:10941800040B43F8040B9142F9D12C492846F9F77B
:10942800EDFA402628482021FBF7EFFE244A049B4A
:109438002749CDE9007605A8FBF7FEFD024640B3B3
:10944800244944F00100F9F7DDFA44F00400224908
:109458000390F9F7D3FA32461B490398F9F710FB42
:109468001E490398F9F7CAFABDF810201449039861
:10947800F9F706FB1A490398F9F7C0FA194903984E
:109488003246F9F7FDFAF9F755F90028FBD105201E
:1094980099E728461449F9F7B1FA012093E70A2019
:1094A80091E700BF746F002038A6070078A6070070
:1094B80019D2070041D2070055D207006CD2070025
:1094C80018730020B8BC07003873002087D2070043
:1094D800D072002098D20700BAD20700C5D2070080
:1094E800CBD207004CB20700D7D207004FF4405345
:1094F8001F4A5B68934213B538D000F500514C6899
:10950800A11A4C424C4193422DD100F500525168AA
:10951800994228D14FF4405316481978142982BF2C
:109528005B691549B3FBF1F3117898BF002314293F
:1095380082BF52691049B2FBF1F21049A0EB010059
:1095480098BF00220E490092C00893424FEA00409B
:109558000C4A40F0030018BF0A460B4914BF012407
:109568000024F9F762FA204602B010BD0024CAE7C9
:10957800DBE5B15178A6070040420F0038A6070086
:10958800E6D20700ECD20700F2D207002DE9F0433B
:10959800ABB006460F4690461C4678222023002191
:1095A8000CA8039300F0B5FF294B1B780BB9FFF704
:1095B800B7FE2CB13146202204A8FBF7FDFD04AE0E
:1095C800244B254C2549DFF8AC90E41AE408240420
:1095D80044F0040543463A462846F9F71CFA03AB1B
:1095E80001933A461E49CDF8009043460CA8FBF774
:1095F80095FD024640B144F001001A49F9F702FA14
:1096080000202BB0BDE8F08320223146484600F008
:1096180020FFD8B1144944F00200F9F7EFF91349D3
:109628002846F9F7EBF9202231462846F9F728FAB7
:109638000F492846F9F7E2F9202249462846F9F762
:109648001FFAF9F777F80028FBD1DAE70120D8E705
:10965800746F002038A6070078A6070032D30700E9
:10966800B8BC070065D3070096D30700B0D307003E
:10967800C2D30700756F002008B5044B986B08B17A
:10968800FFF72EFD024B187008BD00BFF46B0020D9
:109698007873002010B5044658B1B0F5007F0AD899
:1096A800064B00221A70FFF7EFFA054B01209C6366
:1096B80010BD0320FCE70420FAE700BF7873002000
:1096C800F46B002070B5134C0646E06BA36B421890
:1096D8009A420D460BD9104B10481149C01AC008C0
:1096E800000440F00100F9F789F9032070BD5C30EF
:1096F8000A462044314600F0E3FEE36B04F14002E1
:109708002B4429463046E363F9F780FC20640120A6
:10971800ECE700BFF46B002038A6070078A6070026
:10972800D2D30700014B1878704700BF7873002028
:10973800F0B51C4C94F86C2185B07AB394F8D80233
:10974800B4F8DA2204F5377104F5B874164E174DDB
:10975800336800932B68FFF70DFE0128074605D1F3
:10976800201D00F0CBFA0128074614D01048114CF0
:109778001149241AE408240444F00200F9F73EF9D8
:1097880044F004000D490390F9F738F93288296844
:109798000398F9F775F9384605B0F0BD114610463B
:1097A8000434D3E7A46F0020986F00209C6F00203A
:1097B80038A6070078A60700F5D307000BD40700E2
:1097C800334BD3E90E329A422DE9F04106460D4655
:1097D8000DD0304B30483149C01AC008000440F061
:1097E8000100F9F70BF908242046BDE8F0812C4F59
:1097F80097F80080B8F1000F09D0FFF751FB294B0B
:10980800306029461868BDE8F041FFF70BBDFFF747
:1098180067FC80B3FFF78CFF0128C6F80080044678
:10982800C5F8008019D11F4B29461868FFF7FAFCC4
:109838000128044611D1034642462868164D414680
:10984800FFF742FB134BED1AED082D0440B1164902
:1098580045F00100F9F7D2F80424FFF715FAC3E739
:10986800FFF71EFB11493060024645F00400F9F786
:10987800C9F83C70B8E7074B07480D49C01AC0083B
:10988800000440F00100F9F7B9F80524ACE700BF7F
:10989800F46B002038A6070078A6070019D4070043
:1098A800787300207C73002034D407004FD407005D
:1098B8006BD4070037B50D46044630B90749019205
:1098C8004FF42C70F9F7BEFB019A0123294604F1E5
:1098D800720003B0BDE83040FFF758BEC3D107009F
:1098E80013B50446084623781146032B2CD8DFE825
:1098F80003F01402161F0022D4F80140F9F786FB82
:1099080084420AD01448154B1549C01AC0080004EF
:10991800012240F00400F9F775F8012012E00A4628
:1099280000230146601C02B0BDE81040FFF72EBEC0
:10993800034600914022611C0020FFF71BFD431ED7
:109948005842584102B010BD40F2D9300549F9F7E4
:1099580079FB0020F6E700BF78A6070038A60700C5
:1099680088D40700C3D107002DE9F043A3B005460A
:109978000E461446002178221F4604A820239DF88D
:10998800AC800393DDF8A89000F0C3FD41220021CC
:10999800284600F0BEFDB6F89430A34282BF4423A7
:1099A80003FB046393F8968085F80080B8F1030FF1
:1099B80038D8DFE808F009020F2C0022494638465B
:1099C800F9F724FBC5F801004A4639462846FFF74F
:1099D80087FF19E003AB01936B1C009316494B46B4
:1099E8003A4604A8FBF79AFB0028EDD0FAF720FBCB
:1099F800124B1349024613481B1ADB081B0443F099
:109A08000100F8F7FFFF002023B0BDE8F0834421F0
:109A18004C4333199A34B3F898203119681C00F074
:109A28004FFDD1E70548074B0749C01AC008000495
:109A3800424640F00100E4E7B8BC070078A60700FA
:109A4800ABD4070038A60700DCD407002DE9F0479F
:109A5800974B1C68A4B005460F4691460A46014636
:109A68002046FFF727FF002800F0058194F855608D
:109A7800002E38D14FF0010ACDE9007A2B46324644
:109A8800214613A8FFF770FF002800F00F81B9F1F5
:109A9800000F46D0DFF82882412213A908F2A1203E
:109AA80000F00EFD834B84488449C8F82CA0C01AE6
:109AB800C008000440F00400F8F7A0FF94F89230C2
:109AC800C8F8206013B194F8933013B96368C8F8E4
:109AD8000830002239462846F9F798FA784B0124CD
:109AE800C3E90970C2E04122002102A800F011FD7B
:109AF80006F0010A4122002113A806F0020600F030
:109B080008FDBAF1000F40F0C080002E40F0A4809C
:109B18006C4940F26130F9F795FAB9F1000F40F05D
:109B28009E80674B01245C61ABE0A36D03F5FF5297
:109B380003F6FF731F32C3F30B03D31A8A689A42E2
:109B480006D25D485B4B6049C01AC0080004A9E012
:109B58004FF440535A68824213D11A78102A88BFAA
:109B68001A690B7898BF0022102B8CBF0B69002351
:109B78009A4206D050484F4B5449C01AC0080004B6
:109B880090E02846FFF7B2FC88B14B4B494A504950
:109B9800A3EB02084FEAD8084FEA084848F0020049
:109BA800F8F72CFF1EB94B4948F001007CE001236F
:109BB8000193A36D009300222B46214602A8FFF7CC
:109BC800D3FE002872D0CEB1A26DAB18BA1A00210C
:109BD800CDE9002113A852462146FFF7C5FE00280B
:109BE80064D09DF84C304BB13348324B3A49C01AD7
:109BF800C008000440F00200F8F700FFB9F1000FB8
:109C08008FD0BAF1000F2AD02846FFF76FFC10B1A9
:109C18003248FFF727F94122314802A900F050FCE9
:109C2800274B002E14BFAC22A522DA62A26D5A631C
:109C3800002E3FF44EAF2B48412213A900F040FC00
:109C480094F8923023B194F89330002B7FF441AF0D
:109C58001B4B6268DA603CE73A462B46B7E7184B7D
:109C6800AA22DA62E4E72048FFF7FCF8FFF70CF8CD
:109C7800134B9D6405E01724B9F1000FF3D1FFF7EA
:109C880003F8204624B0BDE8F08705F50051174BCE
:109C9800486898423FF449AF0748064B1449C01A30
:109CA800C008000440F00100F8F7A8FE0524E3E727
:109CB8007C73002038A6070078A60700FDD40700AB
:109CC800F46B0020C3D1070076D50700DFD5070065
:109CD8004CD607008DD60700CED607000C6C0020A6
:109CE800546E0020D66E0020186C0020DBE5B151C0
:109CF80025D507000122FFF7A9BE0000F7B50446E5
:109D080018B95D49C420F9F79DF994F85430A3B106
:109D180094F85520032A10D894F86E30032B18D0E5
:109D2800564B57485749C01AC008000440F0010074
:109D3800F8F764FE142003B0F0BD51484F4B524968
:109D4800C01AC008000440F00100F8F757FE0F20C1
:109D5800F1E794F8923023B194F893300BB10120D5
:109D6800E9E7237A33B94648444B4849C01AC00842
:109D78000004E8E7E368342B0BD0404B40484449E3
:109D8800C01AC008000440F00200F8F737FE11209E
:109D9800D1E74FF440553F496868238A88422ED15D
:109DA80043B1616921B3DBB204F114000021CEB2E2
:109DB8009E420BD3314B32483749C01AC0080004C1
:109DC80040F00200F8F71AFE1220B4E750F8047BBE
:109DD800AE89B74201F10101E9D12378B3B9012A6B
:109DE800BDD02748254B2D49C01AC0080004AAE752
:109DF80012B9012BDED1F0E7012AEED1DAE713B16F
:109E08006369002BD6D12378002BD3D01B4B1C4D74
:109E18002349244EED1AED082D0445F003000122D4
:109E28000190F8F7EFFD62681F490198F8F7EAFD1D
:109E3800B2681E490198F8F7E5FD94F85530012BF2
:109E4800636814D8B2680198934203D91849F8F79F
:109E5800D5FD84E701D11749F9E71749F8F7CEFD91
:109E680045F002001549F8F7C9FD102063E7F268CC
:109E780093423FF674AFF3E725D7070038A60700EB
:109E880080A6070096D707007FD70700A9D7070045
:109E9800B8D70700DBE5B151CBD707007AD8070060
:109EA800DBD70700F46B0020DFD70700F2D70700E5
:109EB80015D8070030D807004BD8070066D8070028
:109EC80010DF704711DF704713B50446094968462B
:109ED800FAF75AF8019808B902B010BDD0E9002184
:109EE8002046904718B16846FAF768F8F2E711205B
:109EF800F2E700BFB4D8070013B50446074968461F
:109F0800FAF742F8019B0BB902B010BD2046D3E91D
:109F1800002190476846FAF751F8F3E7CCD80700D4
:109F2800084B9A6822B11A6822F480021A607047B6
:109F3800054B4FF48002C3F88020BFF34F8FBFF367
:109F48006F8F7047443D002000E100E00B4991F815
:109F580016335A09EC231341DB0706D5084B9A68D8
:109F68003AB94FF480030B60704742F20200FBF7E6
:109F7800B5B91A6842F480021A60704700E100E03F
:109F8800443D0020F7B5194F3C7864BB184E0125B5
:109F980020463570FFF798FF112821D02046FFF79B
:109FA800ABFF144B8DF80340186801900DF10300C6
:109FB800F8F7DCFF104901A8FFF782FF0446B0FA62
:109FC80080F0400938709DF80300F8F7FFFF3CB9AE
:109FD8000A4B34701C70FFF7B9FF2846FFF78CFF57
:109FE800204603B0F0BD0824FAE700BF81730020C3
:109FF80080730020ADD80700B95207008273002093
:10A00800F7B5154F3B781BB3144E01203070FFF79E
:10A018005BFF11284FF000051CD00220FFF76CFFF2
:10A028000DF107008DF80750F8F7A0FFFFF74AFF7A
:10A0380004469DF807003D70F8F7C8FF2CB90320C7
:10A048003470FFF76DFFFFF757FF204603B0F0BDF0
:10A058000824FAE72C46F8E7817300208073002073
:10A06800054B1B7833B1054B1B780BB1FFF7C8BF05
:10A07800FFF788BF08207047807300208173002095
:10A08800014B1878704700BF8173002007B5084955
:10A098006846F9F779FF019B13B903B05DF804FB33
:10A0A800D3E9002090476846F9F788FFF3E700BF37
:10A0B800C0D80700FFF7EABF60DF704769DF704765
:10A0C80061DF704730B5134DADF5017D4FF4FA747B
:10A0D8000DF1020103A8ADF80240FFF7F1FF70B9D6
:10A0E800294601A8F9F750FF029B002BF0D003A8DE
:10A0F800D3E90021904701A8F9F760FFF4E70528A4
:10A1080005D00DF5017DBDE83040FBF7E7B80DF54A
:10A11800017D30BD54DB0700024B1B780BB1FFF704
:10A12800D1BF70478373002018B1034B0360002030
:10A1380070470E20704700BFE82A002030B505465A
:10A1480085B00C46002900F0A4800023CDE9013336
:10A15800514A039301230A608DF804008DF80630F4
:10A1680001A906232020ADF80830FFF7A7FF60B14A
:10A17800F9F75EFF494B4A4902464A481B1ADB0871
:10A188001B0443F00100F8F73DFC0023CDE901333F
:10A1980003932268012301A940208DF80530FFF7B9
:10A1A8008DFF60B1F9F744FF3C4B3F4902463D48FB
:10A1B8001B1ADB081B0443F00100F8F723FC0023FB
:10A1C800CDE90133039322688DF80450F72301A9E0
:10A1D8002320ADF80630FFF771FF60B1F9F728FFCB
:10A1E8002E4B324902462F481B1ADB081B0443F04A
:10A1F8000100F8F707FC002301202268039301A956
:10A20800CDE901338DF80400FFF758FF60B1F9F785
:10A218000FFF224B2649024622481B1ADB081B0463
:10A2280043F00100F8F7EEFB0023CDE90233226882
:10A238004FF4B06301A9A1200193FFF73FFF60B17C
:10A24800F9F7F6FE154B1B49024616481B1ADB08A0
:10A258001B0443F00100F8F7D5FB0025226803959D
:10A2680001A9A020CDE90155FFF728FF034668B1F1
:10A27800F9F7DEFE094B104902460A481B1ADB08AB
:10A288001B0443F00100F8F7BDFB2B46184605B048
:10A2980030BD0E23FAE700BFE82A002098A6070081
:10A2A800D8D8070038A607001ED907006AD90700C2
:10A2B800B1D90700FDD907004EDA070073B5054686
:10A2C8000668FFF7F9FE2B68B34204461DD91A4801
:10A2D8001A4B1B491B1ADB081B0443F002000190B0
:10A2E800F8F78CFB2B68174901983246F8F793FB6F
:10A2F8004FF080532A68D3F80C31134901989B0218
:10A3080003F100539A1AF8F77DFB2CB90F4B012281
:10A318001A70204602B070BD2046F9F789FE074B37
:10A328000B49024604481B1ADB081B0443F00100D2
:10A33800F8F768FBEDE700BF38A6070098A6070006
:10A34800A1DA0700D0DA070001DB070083730020D9
:10A358002BDB07004BDF70471FB50E4C01A8FFF73A
:10A36800F9FF70B9214602A8F9F70EFE039B002BEE
:10A37800F4D00198D3E90021904702A8F9F71EFE0E
:10A38800F4E7052804D004B0BDE81040FAF7A6BFEA
:10A3980004B010BD6CDB07007F2805D8034B185CA0
:10A3A800034B5B5C184070470020704784DB070054
:10A3B80004DC0700A0F16103192B98BF203870470F
:10A3C800A0F14103192B98BF203070477F2805D88A
:10A3D800034B185C034B5B5C1840704700207047C8
:10A3E80084DB070004DC0700A0F16103192B98BF88
:10A3F80020387047A0F14103192B98BF20307047CF
:10A408007F299ABF017001206FF02E0070475AB162
:10A418000A787F2A0AD800B10260002119605960C1
:10A42800501A18BF01207047002070476FF02E00A7
:10A438007047000008B5034B5B689B681B6898472A
:10A4480008BD00BF502B002008B50921FFF7F2FF17
:10A4580008BD9AB330B594460F2A18D902460B4660
:10A4680040EA010414F0030F02D00CF1FF3C11E0A4
:10A4780019461046043204330C680568A54206D113
:10A4880010461946ACF1040CBCF1040FF0D8BCF12D
:10A49800010C0FD00A46034684441146184601337E
:10A4A8000132047891F800E0744503D1184611464A
:10A4B8006345F2D100780B78C01A30BD0020704790
:10A4C800844640EA010313F0030F18D18446202A7A
:10A4D8000BD32DE9F007B1E8F807A0E8F807A2F1D7
:10A4E8002002202AF7D2BDE8F007042A07D351F842
:10A4F800043B40F8043BA2F10402042AF7D2002AE4
:10A5080005D011F8013B00F8013B013AF9D160464A
:10A5180070478446002A2DD010F0030F04D000F8AD
:10A52800011B013A26D0F7E7C9B241EA012141EA05
:10A538000141202A12D3A2F120022DE9F0030B4693
:10A548000C460D460E460F4688468946A0E8FA0393
:10A55800203AFBD2BDE8F00320320BD0042A05D301
:10A5680040F8041B043A05D0042AF9D200F8011B6C
:10A57800013AFBD160467047024610F0030F16D12E
:10A5880011F0030F13D12DE9F0004FF001374FF010
:10A59800803351F8044BA4EB070525EA04051D4058
:10A5A80002D142F8044BF4E7A1F10401F0BC11F820
:10A5B800013B02F8013B002BF9D1704700F1010182
:10A5C80010F0030F11D010F8012B002A23D010F03F
:10A5D800030F0AD010F8012B002A1CD010F0030F2B
:10A5E80003D010F8012B002A15D02DE970004FF088
:10A5F80001324FF0803350F8044BA4EB020525EAF2
:10A6080004051D4000D1F6E7A0F1040070BC10F865
:0CA61800012B002AFBD1A0EB01007047D1
:08A62400857F0700457C07005B
:0CA62C000000000003000000DD4E0700ED
:10A6380017A80700000004043BA907000000000059
:10A64800A4BC070000000404ECC3070000000404D5
:10A65800B4C5070000000404E4CA070000000404AD
:10A668002BCE07000000040463CE0700000004049A
:10A6780012D70700000004048ED807000000040465
:10A6880063AA070000000404A5D80700000003031C
:10A6980048DB07000000030360DB0700000003033A
:10A6A800A82B0020702C0020782C0020B02B002034
:10A6B80018000000505400208C6400209D64002085
:08A6C80058540020F4000000CA
:10A6D00048A7070000000000A9A70700102B0020D2
:08A6E000B17607000000000044
:08A6E800353B070000000000F3
:08A6F000F53C0700000000002A
:10A6F80021A107000000000061A30700000000007E
:08A70800E93C0700000000001D
:10A7100000000000000000009D53070000E006005C
:10A72000FFFF060000000000000000004581070058
:08A73000001000000000080009
:10A7380000000000000000000338FDD8704700004A
:10A74800BD23070029240700B9230700433A5C6E9C
:10A758005246355F53444B5F31372E302E325F649B
:10A768003637346464652D315C636F6D706F6E6568
:10A778006E74735C6C69627261726965735C6C6F2C
:10A78800675C7372635C6E72665F6C6F675F64654B
:10A798006661756C745F6261636B656E64732E636A
:10A7A800007274745F6C6F675F6261636B656E647F
:10A7B80000433A5C6E5246355F53444B5F31372E47
:10A7C800302E325F643637346464652D315C636FD4
:10A7D8006D706F6E656E74735C6C696272617269BC
:10A7E80065735C6C6F675C7372635C6E72665F6CDA
:10A7F8006F675F66726F6E74656E642E6300426188
:10A80800636B656E647320666C757368656400615C
:10A8180070700000983C00207F000000183D002068
:10A828001B5B313B33316D0025734C6F67732064BC
:10A83800726F70706564202825642925730D0A00DD
:10A848001B5B306D003C25733E2025733A200020A9
:10A858002530327800202020007C002563001B5B17
:10A86800313B33306D001B5B313B33326D001B5B7A
:10A87800313B33336D001B5B313B33346D001B5B65
:10A88800313B33356D001B5B313B33366D001B5B51
:10A89800313B33376D006572726F72007761726E8B
:10A8A800696E6700696E666F0064656275670000AF
:10A8B80048A8070066A8070028A807006EA8070090
:10A8C80076A807007EA8070086A807008EA80700BC
:10A8D80096A80700000000009EA80700A4A807008B
:10A8E800ACA80700B1A80700433A5C6E5246355F32
:10A8F80053444B5F31372E302E325F643637346421
:10A9080064652D315C636F6D706F6E656E74735C1A
:10A918006C69627261726965735C7574696C5C619B
:10A9280070705F7574696C5F706C6174666F726D5E
:10A938002E63006D656D5F6D6E677200433A5C6EE5
:10A948005246355F53444B5F31372E302E325F64A9
:10A958003637346464652D315C636F6D706F6E6576
:10A968006E74735C6C69627261726965735C626152
:10A978006C6C6F635C6E72665F62616C6C6F632E89
:10A988006300433A5C6E5246355F53444B5F313740
:10A998002E302E325F643637346464652D315C6541
:10A9A800787465726E616C5C667072696E74665CF0
:10A9B8006E72665F667072696E74662E6300433AE3
:10A9C8005C6E5246355F53444B5F31372E302E3222
:10A9D8005F643637346464652D315C6578746572FC
:10A9E8006E616C5C667072696E74665C6E72665FCE
:10A9F800667072696E74665F666F726D61742E63DD
:10AA080000303132333435363738394142434445E2
:10AA180046433A5C6E5246355F53444B5F31372E9E
:10AA2800302E325F643637346464652D315C636F71
:10AA38006D706F6E656E74735C6C69627261726959
:10AA480065735C6673746F726167655C6E72665F6E
:10AA58006673746F726167652E63006E72665F66F7
:10AA680073746F72616765000010000004000000D5
:10AA780001000000CD390700F1390700013A07004D
:10AA8800113A0700653A0700D9390700DD39070090
:10AA9800E139070000100000040000000100000078
:10AAA800793B0700593B0700493B0700853D0700F4
:10AAB800353D07001D3B0700213B0700253B0700EC
:10AAC800433A5C6E5246355F53444B5F31372E3004
:10AAD8002E325F643637346464652D315C636F6D84
:10AAE800706F6E656E74735C6C69627261726965B1
:10AAF800735C6D656D6F626A5C6E72665F6D656DC5
:10AB08006F626A2E6300433A5C6E5246355F534467
:10AB18004B5F31372E302E325F64363734646465CC
:10AB28002D315C636F6D706F6E656E74735C6C69EC
:10AB3800627261726965735C6578706572696D656A
:10AB48006E74616C5F73656374696F6E5F76617252
:10AB5800735C6E72665F73656374696F6E5F697448
:10AB680065722E63004E52465F5355434345535317
:10AB7800004E52465F4552524F525F5356435F480C
:10AB8800414E444C45525F4D495353494E47004E40
:10AB980052465F4552524F525F534F4654444556B2
:10ABA8004943455F4E4F545F454E41424C45440032
:10ABB8004E52465F4552524F525F494E5445524E8F
:10ABC800414C004E52465F4552524F525F4E4F5FC6
:10ABD8004D454D004E52465F4552524F525F4E4FC3
:10ABE800545F464F554E44004E52465F4552524FB1
:10ABF800525F4E4F545F535550504F525445440086
:10AC08004E52465F4552524F525F494E56414C494B
:10AC1800445F504152414D004E52465F4552524F9B
:10AC2800525F494E56414C49445F53544154450084
:10AC38004E52465F4552524F525F494E56414C491B
:10AC4800445F4C454E475448004E52465F45525269
:10AC58004F525F494E56414C49445F464C41475319
:10AC6800004E52465F4552524F525F494E56414C34
:10AC780049445F44415441004E52465F4552524F49
:10AC8800525F444154415F53495A45004E52465F12
:10AC98004552524F525F54494D454F5554004E52FC
:10ACA800465F4552524F525F4E554C4C004E5246ED
:10ACB8005F4552524F525F464F5242494444454EB7
:10ACC800004E52465F4552524F525F494E56414CD4
:10ACD80049445F41444452004E52465F4552524FE8
:10ACE800525F42555359004E52465F4552524F5299
:10ACF8005F434F4E4E5F434F554E54004E52465F92
:10AD08004552524F525F5245534F55524345530097
:10AD18004E52465F4552524F525F4D4F44554C4537
:10AD28005F4E4F545F494E495449414C495A454436
:10AD3800004E52465F4552524F525F4D555445584A
:10AD48005F494E49545F4641494C4544004E52467E
:10AD58005F4552524F525F4D555445585F4C4F43D3
:10AD68004B5F4641494C4544004E52465F4552525E
:10AD78004F525F4D555445585F554E4C4F434B5FAE
:10AD88004641494C4544004E52465F4552524F5247
:10AD98005F4D555445585F434F4E445F494E4954A3
:10ADA8005F4641494C4544004E52465F4552524F1A
:10ADB800525F4D4F44554C455F414C5245414459B3
:10ADC8005F494E495449414C495A4544004E524600
:10ADD8005F4552524F525F53544F524147455F4669
:10ADE800554C4C004E52465F4552524F525F4150AF
:10ADF800495F4E4F545F494D504C454D454E544563
:10AE080044004E52465F4552524F525F46454154A8
:10AE18005552455F4E4F545F454E41424C454400A4
:10AE28004E52465F4552524F525F494F5F50454E12
:10AE380044494E47004E52465F4552524F525F4476
:10AE480052565F5457495F4552525F4F56455252CA
:10AE5800554E004E52465F4552524F525F4452562D
:10AE68005F5457495F4552525F414E41434B004E34
:10AE780052465F4552524F525F4452565F545749AB
:10AE88005F4552525F444E41434B004E52465F4528
:10AE980052524F525F424C455F495053505F52588F
:10AEA8005F504B545F5452554E4341544544004EF5
:10AEB80052465F4552524F525F424C455F4950538C
:10AEC800505F4348414E4E454C5F414C52454144CA
:10AED800595F455849535453004E52465F455252A4
:10AEE8004F525F424C455F495053505F4C494E4B5F
:10AEF8005F444953434F4E4E4543544544004E52D8
:10AF0800465F4552524F525F424C455F495053503D
:10AF18005F504545525F52454A45435445440055A4
:10AF28006E6B6E6F776E206572726F7220636F64DE
:10AF380065000000000000006DAB07000100000084
:10AF480079AB07000200000097AB07000300000080
:10AF5800B8AB070004000000CBAB070005000000F9
:10AF6800DCAB070006000000F0AB0700070000009C
:10AF780008AC07000800000020AC0700090000002A
:10AF880038AC07000A00000051AC07000B000000B5
:10AF980069AC07000C00000080AC07000D00000041
:10AFA80094AC07000E000000A6AC07000F000000DC
:10AFB800B5AC070010000000C9AC07001100000084
:10AFC800E0AC070012000000EFAC0700130000001F
:10AFD80004AD07008000000018AD070081000000E4
:10AFE80039AD07008200000055AD0700830000005E
:10AFF80071AD0700840000008FAD070085000000D8
:10B00800B0AD070086000000D5AD07009000000035
:10B01800ECAD0700910000000AAE070092000000A6
:10B0280028AE0700008200003DAE07000182000044
:10B038005BAE07000282000077AE070000840000C4
:10B0480093AE070001840000B7AE07000284000039
:10B05800E1AE07000384000006AF0700982F8A427C
:10B0680091443771CFFBC0B5A5DBB5E95BC2563952
:10B07800F111F159A4823F92D55E1CAB98AA07D86A
:10B08800015B8312BE853124C37D0C55745DBE728D
:10B09800FEB1DE80A706DC9B74F19BC1C1699BE40D
:10B0A8008647BEEFC69DC10FCCA10C246F2CE92D9D
:10B0B800AA84744ADCA9B05CDA88F97652513E98C1
:10B0C8006DC631A8C82703B0C77F59BFF30BE0C6C8
:10B0D8004791A7D55163CA0667292914850AB72756
:10B0E80038211B2EFC6D2C4D130D385354730A65F3
:10B0F800BB0A6A762EC9C281852C7292A1E8BFA2CA
:10B108004B661AA8708B4BC2A3516CC719E892D131
:10B11800240699D685350EF470A06A1016C1A419B4
:10B12800086C371E4C774827B5BCB034B30C1C39B3
:10B138004AAAD84E4FCA9C5BF36F2E68EE828F7472
:10B148006F63A5781478C8840802C78CFAFFBE908C
:10B15800EB6C50A4F7A3F9BEF27871C6480028003A
:10B1680000204000616107001D480700C347070031
:10B17800134D0700834D0700A34D07001347070031
:10B18800D5460700AF4C0700000000002E2E2F2EDA
:10B198002E2F2E2E2F2E2E2F2E2E2F6D6F64756C88
:10B1A80065732F6E7266782F68616C2F6E72665F9A
:10B1B8006770696F2E6800433A5C6E5246355F537C
:10B1C800444B5F31372E302E325F64363734646437
:10B1D800652D315C636F6D706F6E656E74735C6244
:10B1E8006F617264735C626F617264732E63000BCB
:10B1F8000C18190D0E0F10433A5C6E5246355F530A
:10B20800444B5F31372E302E325F643637346464F6
:10B21800652D315C636F6D706F6E656E74735C6CF9
:10B2280069627261726965735C63727970746F5C6C
:10B238006E72665F63727970746F5F73686172654E
:10B24800642E6300AAF3E1DA9E0508BD14A972B161
:10B25800CCFEACD22CAA2B883A3C21E96F541C2D89
:10B26800B50A9E516F11FEF684EDE4D83F99B4D427
:10B27800D43BD4AC6C734ECDE5FA90770E9B30BEC0
:10B288006D9C819A52656365697665642061206664
:10B2980061756C74212069643A20307825303878DB
:10B2A8002C2070633A203078253038782C20696E4D
:10B2B800666F3A20307825303878005265636569C2
:10B2C80076656420616E206572726F723A203078FC
:10B2D800253038782100496E73696465206D61698D
:10B2E8006E004166746572206D61696E2C2073680A
:10B2F8006F756C64206E6576657220626520726574
:10B3080061636865642E00000338FDD870472D2DF1
:10B318003E204576656E742072656365697665645E
:10B328003A204552524F52207768696C65206578FB
:10B3380065637574696E6720616E206673746F72D9
:10B34800616765206F7065726174696F6E2E002D7C
:10B358002D3E204576656E74207265636569766555
:10B36800643A2077726F7465202564206279746569
:10B37800732061742061646472657373203078256A
:10B38800782E002D2D3E204576656E7420726563FB
:10B3980065697665643A2065726173656420256421
:10B3A80020706167652066726F6D206164647265E4
:10B3B800737320307825782E0000000008200001E3
:10B3C800FFFFFFFFFFFFFFFFFFFFFFFF0000000081
:10B3D800000000000000000001000000FFFFFFFF68
:10B3E800512563FCC2CAB9F3849E17A7ADFAE6BC1F
:10B3F800FFFFFFFFFFFFFFFF00000000FFFFFFFF51
:10B4080096C298D84539A1F4A033EB2D817D0377F6
:10B41800F240A463E5E6BCF847422CE1F2D1176B91
:10B42800F551BF376840B6CBCE5E316B5733CE2B64
:10B43800169E0F7C4AEBE78E9B7F1AFEE242E34F93
:10B448004B60D2273E3CCE3BF6B053CCB0061D65D0
:10B45800BC86987655BDEBB3E7933AAAD835C65A59
:10B46800335B0700855C0700E95C07005465726D73
:10B47800696E616C00525454005345474745520069
:10B48800526573657474696E6720626F6F746C6F50
:10B49800616465722E00496E6163746976697479B6
:10B4A8002074696D656F75742E00696E207765610B
:10B4B8006B206E72665F6466755F696E69745F752E
:10B4C80073657200496E206E72665F626F6F746C8E
:10B4D8006F616465725F696E697400426F6F742092
:10B4E80076616C69646174696F6E206661696C6508
:10B4F800642E204E6F2076616C6964206170702024
:10B50800746F20626F6F742E00426F6F74207661C3
:10B518006C69646174696F6E206661696C65642E1C
:10B5280020536F667444657669636520697320707B
:10B53800726573656E742062757420696E76616CCD
:10B5480069642E00426F6F742076616C696461745F
:10B55800696F6E206661696C65642E204170702089
:10B56800697320696E76616C69642E004170702081
:10B5780069732076616C696400444655206D6F6478
:10B5880065206265636175736520617070206973F9
:10B59800206E6F742076616C69642E0044465520D5
:10B5A8006D6F646520726571756573746564207666
:10B5B800696120627574746F6E2E00444655206D63
:10B5C8006F6465207265717565737465642076694A
:10B5D800612047505245475245542E00556E7265BA
:10B5E80061636861626C6500456E746572206D61A7
:10B5F800696E206C6F6F7000433A5C6E5246355F1F
:10B6080053444B5F31372E302E325F643637346403
:10B6180064652D315C636F6D706F6E656E74735CFD
:10B628006C69627261726965735C626F6F746C6F6A
:10B63800616465725C6E72665F626F6F746C6F6175
:10B648006465722E630052756E6E696E67206E7245
:10B65800665F626F6F746C6F616465725F61707052
:10B668005F737461727420776974682061646472AE
:10B678006573733A203078253038780044697361EF
:10B68800626C696E6720696E746572727570747326
:10B698002E204E5649432D3E494345525B305D3A74
:10B6A8002030782578004661696C65642072756E73
:10B6B8006E696E67206E72665F6466755F6D627232
:10B6C8005F6972715F666F72776172645F616464EB
:10B6D800726573735F736574282900436F756C64B2
:10B6E800206E6F742070726F7465637420626F6F60
:10B6F800746C6F6164657220616E64207365747424
:10B70800696E67732070616765732C2030782578BF
:10B718002E00436F756C64206E6F742070726F74A6
:10B7280065637420536F6674446576696365206148
:10B738006E64206170706C69636174696F6E2C202F
:10B74800307825782E00433A5C6E5246355F534474
:10B758004B5F31372E302E325F6436373464646580
:10B768002D315C636F6D706F6E656E74735C6C69A0
:10B77800627261726965735C626F6F746C6F616429
:10B7880065725C6E72665F626F6F746C6F61646520
:10B79800725F6170705F73746172745F66696E6105
:10B7A8006C2E630074696D65725F6163746976619C
:10B7B80074652028307825782900433A5C6E524613
:10B7C800355F53444B5F31372E302E325F64363746
:10B7D800346464652D315C636F6D706F6E656E7473
:10B7E800735C6C69627261726965735C626F6F74B5
:10B7F8006C6F616465725C6E72665F626F6F746CA9
:10B808006F616465725F6466755F74696D65727394
:10B818002E630074696D65725F73746F70202830D1
:10B82800782578290074696D65725F66697265208C
:10B8380028307825782900000338FDD870475665E8
:10B8480072696679696E6720424C3A204164647275
:10B858003A203078253038782C205372633A2030DB
:10B8680078253038782C204C656E3A203078253091
:10B878003878004E6F20626F6F746C6F6164657208
:10B8880020636F7079206E65656465642C20626F33
:10B898006F746C6F61646572207570646174652083
:10B8A800636F6D706C6574652E00436F7079696E97
:10B8B8006720626F6F746C6F616465723A205372AF
:10B8C800633A203078253038782C204C656E3A2041
:10B8D8003078253038780052657175657374207436
:10B8E8006F20636F707920424C206661696C6564D3
:10B8F800004E6F20636F7079206E65656465640023
:10B90800433A5C6E5246355F53444B5F31372E30B5
:10B918002E325F643637346464652D315C636F6D35
:10B92800706F6E656E74735C6C6962726172696562
:10B93800735C626F6F746C6F616465725C6E726663
:10B948005F626F6F746C6F616465725F66775F6169
:10B95800637469766174696F6E2E6300436F7079E2
:10B96800696E67203078257820746F2030782578C4
:10B978002C2073697A653A20307825780046616909
:10B988006C656420746F20777269746520696D61D5
:10B99800676520636F7079696E672070726F677270
:10B9A80065737320746F2073657474696E67732090
:10B9B800706167652E00456E746572206E72665FF1
:10B9C800626F6F746C6F616465725F6466755F73D4
:10B9D800645F636F6E74696E756500536F7572632B
:10B9E80065206164647265737320646F6573206E8B
:10B9F8006F7420636F6E7461696E20612076616C6C
:10BA0800696420536F66744465766963652E0053D4
:10BA18004420616C726561647920636F7069656444
:10BA2800005570646174696E672053442E204F6C12
:10BA380064205344207665723A2025642C204E6594
:10BA480077207665723A202564004661696C6564E2
:10BA580020746F20636F7079206669726D776172E8
:10BA6800652E00456E746572206E72665F626F6F38
:10BA7800746C6F616465725F66775F616374697621
:10BA88006174650056616C69642041707000456E90
:10BA9800746572206E72665F6466755F6170705F50
:10BAA800636F6E74696E75650053657474696E674B
:10BAB800206170702061732076616C696400435264
:10BAC8004320636F6D7075746174696F6E20666171
:10BAD800696C656420666F7220636F7069656420A5
:10BAE8006170703A20737263206372633A20307811
:10BAF800253038782C20726573206372633A2030C1
:10BB080078253038780056616C69642053440056B3
:10BB1800616C696420424C0056616C69642053442E
:10BB2800202B20424C00456E746572206E72665F51
:10BB38006466755F73645F626C5F636F6E74696E71
:10BB480075650053442B424C3A20534420636F7070
:10BB580079206661696C65640053442B424C3A2035
:10BB6800424C20636F7079206661696C6564004E91
:10BB78006F206669726D7761726520746F206163EA
:10BB88007469766174652E004163746976617469BD
:10BB98006F6E206661696C656420776974682065DA
:10BBA80072726F72202564202862616E6B20636F49
:10BBB80064653A203078257829004120536F6674EF
:10BBC80044657669636520686173206A75737420BB
:10BBD8006265656E206163746976617465642E20A0
:10BBE80049742773206C696B656C7920746861747B
:10BBF80020616E206170706C69636174696F6E207A
:10BC080077696C6C20636F6D6520696D6D6564691B
:10BC18006174656C7900436F756C64206E6F742075
:10BC280077726974652073657474696E67732E0022
:10BC3800496E7465726E616C206665656400574470
:10BC48005420656E61626C6564204352563A2564DF
:10BC5800207469636B73005374617274696E672032
:10BC6800612074696D657220282564207469636B8E
:10BC7800732920666F722066656564696E67207730
:10BC880061746368646F672E005744542069732099
:10BC98006E6F7420656E61626C6564006E72665FBB
:10BCA800626F6F746C6F616465725F7764740000B3
:10BCB800D3740700CD740700AD740700200000009E
:10BCC80078000000000000000100010000000000F2
:10BCD8000100000000000000020005000100000053
:10BCE800420000000000000000000000000000000A
:10BCF8000000000000000000010011000100FFFF2B
:10BD08000100000000000000020017000200FEFF12
:10BD18006401000060BD0700000000000000000092
:10BD28000000000000000000010001000000000009
:10BD380001000000000000000200050001000000F2
:10BD480022000000000000000000000000000000C9
:10BD58000000000000000000010011000400FCFFCA
:10BD68000400000000000000020011000400FCFFB5
:10BD78000400000000000000030021000400FCFF94
:10BD88000400100000000000040011000100FFFF83
:10BD98000100000000000000050011000200FEFF85
:10BDA8000400000000000000060011000400FCFF71
:10BDB8000400000000000000070011000400FCFF60
:10BDC8000400000000000000080017000200FEFF49
:10BDD8002400000030BD0700090010000100FFFF2B
:10BDE8000100000010BE07000A0027000200FEFF45
:10BDF80044000300D0BC0700000000000000000061
:10BE08000000000000000000000000000100170012
:10BE18000400FCFF6801000000BD070002001700D5
:10BE28000400FCFFAC01000044BE07000000000055
:10BE380000000000000000000000000001000700F2
:10BE4800000000006801000000BD070002000100BA
:10BE580000000000010000000000000003000500D1
:10BE68000100000042000000000000000000000087
:10BE7800000000000000000000000000456E74652E
:10BE880072696E6720444655206D6F64652E0043C5
:10BE98006F756C64206E6F7420696E6974616C696B
:10BEA8007A6520444655207472616E73706F72749F
:10BEB8003A203078253038780046726565696E67B3
:10BEC8002062756666657220257000416476657229
:10BED800746973696E672E2E2E00436F6E6E6563EC
:10BEE800746564004661696C75726520746F2075AD
:10BEF800706461746520636F6E6E656374696F6EDC
:10BF080020706172616D65746572733A20307825AE
:10BF1800780063616E6E6F7420616C6C6F6361741E
:10BF280065206D656D6F7279206275666665722130
:10BF380000427566666572202570206163717569B7
:10BF48007265642C206C656E202564202825642980
:10BF580000526563656976656420424C455F4741D8
:10BF68005454535F4556545F45584348414E4745DE
:10BF78005F4D54555F5245515545535420287265BD
:10BF880071756573743A2025642C207265706C791C
:10BF98003A202564292E0052656365697665642018
:10BFA800424C455F4741505F4556545F44415441B8
:10BFB8005F4C454E4754485F5550444154455F5285
:10BFC8004551554553542E0052656365697665643D
:10BFD80020424C455F4741505F4556545F444154A9
:10BFE800415F4C454E4754485F55504441544520A5
:10BFF8002825752C206D61785F72785F74696D658E
:10C00800202575292E00526563656976656420428E
:10C018004C455F4741505F4556545F5345435F5019
:10C028004152414D535F5245515545535400434386
:10C03800434420666F722073657276696365206376
:10C0480068616E67656420697320307825303478BC
:10C0580000526563656976656420424C455F4741D7
:10C06800505F4556545F434F4E4E5F504152414DCD
:10C078005F555044415445006D61785F636F6E6E43
:10C088005F696E74657276616C3A202564006D692B
:10C098006E5F636F6E6E5F696E74657276616C3A1F
:10C0A80020256400736C6176655F6C6174656E63EE
:10C0B800793A20256400636F6E6E5F7375705F74E4
:10C0C800696D656F75743A2025640052656365690A
:10C0D80076656420424C455F4741505F4556545F42
:10C0E800434F4E4E5F504152414D5F55504441546D
:10C0F800455F52455155455354004661696C757208
:10C108006520746F2075706461746520636F6E6E4E
:10C11800656374696F6E20706172616D65746572B4
:10C1280020726571756573743A20307825780052ED
:10C138006563656976656420424C455F4741505F99
:10C148004556545F5048595F55504441544520283E
:10C1580052583A25642C2054583A25642C2073747C
:10C16800617475733A25642900526563656976655B
:10C178006420424C455F4741505F4556545F5048E4
:10C18800595F5550444154455F52455155455354A4
:10C198002E005365742072656365697074206E6F34
:10C1A80074696600436F756C64206E6F74206861F3
:10C1B8006E646C65206F6E5F6374726C5F70745F21
:10C1C80077726974652E206572725F636F64653A71
:10C1D8002030782530347800526563656976656467
:10C1E80020424C455F4741505F4556545F53454395
:10C1F8005F494E464F5F5245515545535400466975
:10C208006E69736865642068616E646C696E672026
:10C21800636F6E6E2073656320757064617465006A
:10C228005368757474696E6720646F776E20424C2A
:10C2380045207472616E73706F72742E0044697356
:10C24800636F6E6E656374696E672E00424C45209D
:10C258007472616E73706F72742073687574206481
:10C268006F776E2E00433A5C6E5246355F53444BEF
:10C278005F31372E302E325F643637346464652D73
:10C28800315C636F6D706F6E656E74735C6C696240
:10C298007261726965735C626F6F746C6F616465FB
:10C2A800725C626C655F6466755C6E72665F64661C
:10C2B800755F626C652E6300444655207265717522
:10C2C800657374202564206661696C6564207769EC
:10C2D8007468206572726F723A2030782578004948
:10C2E8006E697469616C697A696E6720424C452091
:10C2F800444655207472616E73706F727400536592
:10C308007474696E6720757020766563746F722027
:10C318007461626C653A2030782530387800456E53
:10C3280061626C696E6720536F66744465766963F1
:10C33800652E00436F6E6669677572696E67204285
:10C348004C4520737461636B2E00456E61626C69A5
:10C358006E672074686520424C4520737461636B76
:10C368002E004E6F206164766572746973696E671A
:10C37800206E616D6520666F756E64005365747418
:10C38800696E6720616476206E616D653A20257359
:10C398002C206C656E6774683A20256400557369B3
:10C3A8006E672064656661756C7420616476657279
:10C3B800746973696E67206E616D650052336368D6
:10C3C8006172676500424C4520444655207472618D
:10C3D8006E73706F727420696E697469616C697AC2
:10C3E80065642E006E72665F6466755F626C6500D8
:10C3F80050EADA308883B89F604F15F30000C98E81
:10C4080000000000000000000338FDD870470C0051
:10C418000C000000580277726974650065726173D8
:10C428006500466C617368202573207375636365C6
:10C4380073733A20616464723D25702C2070656EB8
:10C4480064696E6720256400466C617368202573F3
:10C45800206661696C6564202830782578293A203F
:10C46800616464723D25702C206C656E3D307825C2
:10C47800782062797465732C2070656E64696E67C4
:10C4880020256400496E697469616C697A696E6710
:10C49800206E72665F6673746F726167655F73643E
:10C4A800206261636B656E642E00496E6974696110
:10C4B8006C697A696E67206E72665F6673746F72F4
:10C4C8006167655F6E766D63206261636B656E643C
:10C4D8002E006E72665F6673746F726167655F7750
:10C4E8007269746528616464723D25702C207372CA
:10C4F800633D25702C206C656E3D2564206279743F
:10C508006573292C2071756575652075736167657C
:10C518003A202564006E72665F6673746F72616795
:10C52800655F77726974652829206661696C65643E
:10C538002077697468206572726F72203078257868
:10C548002E006E72665F6673746F726167655F65F1
:10C558007261736528616464723D307825702C209F
:10C568006C656E3D2564207061676573292C2071A8
:10C57800756575652075736167653A202564006E79
:10C5880072665F6673746F726167655F6572617307
:10C59800652829206661696C65642077697468205C
:10C5A8006572726F7220307825782E006E72665F21
:10C5B8006466755F666C61736800416C6C20666CBC
:10C5C800617368206F7065726174696F6E7320683B
:10C5D80061766520636F6D706C657465642E2044A8
:10C5E800465520636F6D706C657465642E004661F6
:10C5F800696C656420746F207363686564756C6525
:10C60800206F626A65637420657865637574653A3E
:10C6180020307825782E0057686F6C65206669721F
:10C628006D7761726520696D616765207265636504
:10C63800697665642E20506F737476616C696461E5
:10C6480074696E672E005265717565737420686130
:10C658006E646C696E6720636F6D706C6574652EAF
:10C6680020526573756C743A203078257800433A07
:10C678005C6E5246355F53444B5F31372E302E3255
:10C688005F643637346464652D315C636F6D706F39
:10C698006E656E74735C6C69627261726965735CF5
:10C6A800626F6F746C6F616465725C6466755C6EF2
:10C6B80072665F6466755F7265715F68616E646CEF
:10C6C80065722E630048616E646C65204E52465F49
:10C6D8004446555F4F505F524543454950545F4E5D
:10C6E8004F5449465F5345540048616E646C652059
:10C6F8004E52465F4446555F4F505F41424F525439
:10C708000048616E646C65204E52465F4446555F32
:10C718004F505F4F424A4543545F43524541544549
:10C728002028636F6D6D616E64290048616E646CCA
:10C7380065204E52465F4446555F4F505F43524313
:10C748005F4745542028636F6D6D616E642900480A
:10C75800616E646C65204E52465F4446555F4F508B
:10C768005F4F424A4543545F575249544520286316
:10C778006F6D6D616E64290048616E646C65204E52
:10C7880052465F4446555F4F505F4F424A454354B7
:10C798005F455845435554452028636F6D6D616E5C
:10C7A80064290057726974696E672076616C6964E0
:10C7B80020696E697420636F6D6D616E6420746F9B
:10C7C80020666C6173682E0048616E646C65204E4B
:10C7D80052465F4446555F4F505F4F424A45435467
:10C7E8005F53454C4543542028636F6D6D616E64FB
:10C7F800290048616E646C65204E52465F44465578
:10C808005F4F505F4F424A4543545F43524541543E
:10C8180045202864617461290043616E6E6F74203D
:10C828006372656174652064617461206F626A6512
:10C83800637420776974686F75742076616C6964B5
:10C8480020696E697420636F6D6D616E64004F625C
:10C858006A6563742073697A652063616E6E6F74AC
:10C8680020626520302E004F626A65637420736908
:10C878007A65206D75737420626520706167652024
:10C88800616C69676E656400496E76616C696420E5
:10C8980073697A6520666F72206F626A65637420B7
:10C8A80028746F6F206C6172676529004372656137
:10C8B80074696E6720746865206F626A65637420A6
:10C8C800776974682073697A6520307825303878FC
:10C8D80020776F756C64206F766572666C6F772051
:10C8E8006669726D776172652073697A652E204F6B
:10C8F800666673657420697320307825303878202F
:10C90800616E64206669726D776172652073697AF9
:10C9180065206973203078253038782E004572619B
:10C928007365206F7065726174696F6E20666169E6
:10C938006C6564004372656174696E67206F626A32
:10C9480065637420776974682073697A653A20256D
:10C95800642E204F66667365743A20307825303827
:10C96800782C204352433A203078253038780048D4
:10C97800616E646C65204E52465F4446555F4F5069
:10C988005F4F424A4543545F5752495445202864F3
:10C9980061746129005772697465207265717565E3
:10C9A800737420746F6F206C6F6E670048616E64DB
:10C9B8006C65204E52465F4446555F4F505F435268
:10C9C800435F47455420286461746129004F6666B7
:10C9D8007365743A25642C204352433A30782530E5
:10C9E80038780048616E646C65204E52465F444654
:10C9F800555F4F505F4F424A4543545F4558454342
:10CA08005554452028646174612900496E76616C2B
:10CA1800696420646174612E20657870656374654B
:10CA2800643A2025642C20676F743A2025640048F6
:10CA3800616E646C65204E52465F4446555F4F50A8
:10CA48005F4F424A4543545F53454C454354202861
:10CA5800646174612900637263203D203078257811
:10CA68002C206F6666736574203D20307825782CFD
:10CA7800206D61785F73697A65203D20307825786C
:10CA880000496E76616C6964206F626A6563742020
:10CA98007479706520696E20726571756573742E7E
:10CAA80000496E76616C6964206F70636F646520FD
:10CAB80072656365697665643A20307825782E005A
:10CAC8005363686564756C65722072616E206F755A
:10CAD80074206F6620737061636521006E72665FF3
:10CAE8006466755F7265715F68616E646C6572001B
:10CAF80044657374696E6174696F6E2073657474CC
:10CB0800696E677320617265206964656E74696314
:10CB1800616C20746F20736F757263652C20777257
:10CB2800697465206E6F74206E65656465642E2077
:10CB3800536B697070696E672E0057726974696EFD
:10CB4800672073657474696E67732E2E2E004572A4
:10CB58006173696E67206F6C642073657474696EA5
:10CB680067732061743A2030782530387800436F35
:10CB7800756C64206E6F74206572617365207468CB
:10CB8800652073657474696E6773207061676521C9
:10CB980000436F756C64206E6F74207772697465DA
:10CBA80020746865204446552073657474696E67FF
:10CBB80073207061676521005573696E672073651E
:10CBC8007474696E677320706167652E00436F70B7
:10CBD80079696E6720666F7262696464656E207039
:10CBE800617274732066726F6D206261636B757019
:10CBF80020706167652E00526573746F72696E6785
:10CC08002073657474696E67732066726F6D206235
:10CC180061636B75702073696E6365207468652045
:10CC280073657474696E6773207061676520636FDC
:10CC38006E74656E74732061726520696E76616CBE
:10CC480069642028435243206572726F72292E004E
:10CC5800526573657474696E6720626F6F746C6F68
:10CC6800616465722073657474696E677320736993
:10CC78006E6365206E6569746865722074686520E6
:10CC880073657474696E67732070616765206E6F71
:10CC98007220746865206261636B757020617265CB
:10CCA8002076616C69642028435243206572726F54
:10CCB80072292E004F6C642073657474696E6773F3
:10CCC80020706167652064657465637465642E20EF
:10CCD800557067726164696E6720696E666F2E00B1
:10CCE8004261636B696E672075702073657474693F
:10CCF8006E6773207061676520746F206164647269
:10CD080065737320307825782E00433A5C6E52465E
:10CD1800355F53444B5F31372E302E325F643637E0
:10CD2800346464652D315C636F6D706F6E656E740D
:10CD3800735C6C69627261726965735C626F6F744F
:10CD48006C6F616465725C6466755C6E72665F6464
:10CD580066755F73657474696E67732E6300436FDD
:10CD6800756C64206E6F7420706572666F726D20CA
:10CD78006261636B7570206F6620626F6F746C6F91
:10CD8800616465722073657474696E6773212045E8
:10CD980072726F723A20307825780043616C6C6942
:10CDA8006E67206E72665F6466755F73657474691A
:10CDB8006E67735F696E697428292E2E2E006E7255
:10CDC800665F6466755F666C6173685F696E6974D7
:10CDD8002829206661696C65642077697468206514
:10CDE80072726F723A202578006E72665F6466759B
:10CDF8005F73657474696E67735F77726974655F72
:10CE0800616E645F6261636B757028292066616971
:10CE18006C65642077697468206572726F723A2055
:10CE28002578006E72665F6466755F7365747469F1
:10CE38006E67730045726173696E672073657474F9
:10CE4800696E6773207061676520616464697469DD
:10CE58006F6E616C20646174612E006E72665F642F
:10CE680066755F73657474696E67735F73766369FB
:10CE780000496E697469616C697A696E67207472B9
:10CE8800616E73706F7274732028666F756E643A82
:10CE980020256429004661696C656420746F2069E7
:10CEA8006E697469616C697A65207472616E7370F9
:10CEB8006F72742025642C206572726F722025644D
:10CEC800005368757474696E6720646F776E207498
:10CED80072616E73706F7274732028666F756E64FA
:10CEE8003A20256429004661696C656420746F20C6
:10CEF80073687574646F776E207472616E73706F87
:10CF080072742025642C206572726F72202564006B
:10CF1800456E746572206E72665F6466755F6361E4
:10CF28006368655F70726570617265282900726553
:10CF38007175697265645F73697A653A203078251E
:10CF4800782E00747275650066616C73650073698C
:10CF58006E676C655F62616E6B3A2025732E006B9D
:10CF68006565705F6170703A2025732E006B65658A
:10CF7800705F736F66746465766963653A202573BC
:10CF88002E0053445F50524553454E543A20257362
:10CF98002E0042616E6B20636F6E74656E74733A17
:10CFA8000042616E6B203020636F64653A203078F0
:10CFB800253032783A2053697A653A2030782578D6
:10CFC8000042616E6B203120636F64653A203078CF
:10CFD800253032783A2053697A653A2030782578B6
:10CFE80000433A5C6E5246355F53444B5F31372EEF
:10CFF800302E325F643637346464652D315C636F7C
:10D008006D706F6E656E74735C6C69627261726963
:10D0180065735C626F6F746C6F616465725C646683
:10D02800755C6E72665F6466755F7574696C732E85
:10D038006300706173733A2025642E00636163682E
:10D04800655F616464726573733A20307825782E61
:10D058000063616368655F746F6F5F736D616C6CAB
:10D068003A2025732E006B6565705F6669726D776F
:10D078006172653A2025732E0064656C6574655F7E
:10D088006D6F72653A2025732E0041626F72746964
:10D098006E672E2043616E6E6F7420666974206E11
:10D0A8006577206669726D77617265206F6E20649E
:10D0B800657669636500496E76616C696461746957
:10D0C8006E67206170702E0048616E646C65723AFC
:10D0D80020496E76616C69642070726F746F636F3B
:10D0E8006C20627566666572206D5F70625F73742E
:10D0F8007265616D0048616E646C65723A20496EB4
:10D1080076616C696420696E697420636F6D6D6106
:10D118006E642E0048616E646C65723A20496E76C2
:10D12800616C69642070726F746F636F6C206275D4
:10D1380066666572206D5F70625F73747265616D9B
:10D148002028696E697420636F6D6D616E642900B3
:10D15800424C2073697A652028256429206F7665FA
:10D1680072206C696D6974202825642900496E69EC
:10D1780074207061636B657420646F6573206E6FD3
:10D188007420636F6E7461696E2076616C696420C7
:10D198006669726D776172652073697A65005042BD
:10D1A8003A20496E6974207061636B65742064610C
:10D1B8007461206C656E3A20256400433A5C6E52B7
:10D1C80046355F53444B5F31372E302E325F64361D
:10D1D80037346464652D315C636F6D706F6E656E96
:10D1E80074735C6C69627261726965735C626F6F9B
:10D1F800746C6F616465725C6466755C6E72665FA0
:10D208006466755F76616C69646174696F6E2E63BC
:10D21800005369676E61747572652072657175690E
:10D228007265642E20436865636B696E6720736955
:10D23800676E61747572652E004E6F207369676E34
:10D24800617475726520666F756E642E00496E761E
:10D25800616C6964207369676E61747572652074A6
:10D268007970650043616C63756C6174696E6720E1
:10D278006861736820286C656E3A20256429005619
:10D288006572696679207369676E61747572650085
:10D298005369676E6174757265206661696C65644F
:10D2A80020286572725F636F64653A20307825784C
:10D2B80029005369676E61747572653A0048617335
:10D2C800683A005075626C6963204B65793A004989
:10D2D8006D616765207665726966696564006D6170
:10D2E8006A6F72006D696E6F7200536F6674446581
:10D2F800766963652075706461746520697320615F
:10D308002025732076657273696F6E20757064616D
:10D3180074652E2043757272656E743A2025642EEA
:10D32800204E65773A2025642E0048617368207680
:10D338006572696669636174696F6E2E20737461C2
:10D34800727420616464726573733A20307825784A
:10D358002C2073697A653A203078257800436F75F8
:10D368006C64206E6F742072756E2068617368201B
:10D37800766572696669636174696F6E2028657283
:10D38800725F636F64652030782578292E004861C4
:10D39800736820766572696669636174696F6E2067
:10D3A8006661696C65642E004578706563746564B0
:10D3B80020465720686173683A0041637475616C50
:10D3C80020465720686173683A00496E6974206383
:10D3D8006F6D6D616E64206C617267657220746830
:10D3E800616E2065787065637465642E005072659F
:10D3F80076616C69646174696F6E206661696C65D9
:10D40800642E00496E697420636F6D6D616E643AB5
:10D41800004578656375746520776974682066616E
:10D42800756C7479206F66667365740043616E2746
:10D43800742066696E6420726F6F6D20666F72204B
:10D4480075706461746500577269746520616464FD
:10D45800726573732073657420746F20307825307B
:10D468003878004661696C656420746F2064656370
:10D478006F646520696E6974207061636B65740000
:10D4880043524320636865636B206F662061707048
:10D49800206661696C65642E2052657475726E2011
:10D4A8002564006E72665F63727970746F5F68617D
:10D4B80073685F63616C63756C61746528292066A5
:10D4C80061696C65642077697468206572726F722F
:10D4D80020257300496E76616C696420626F6F74F1
:10D4E8002076616C69646174696F6E207479706507
:10D4F8003A20256400496E76616C69646174696ECE
:10D5080067206F6C64206170706C69636174696F07
:10D518006E20696E2062616E6B20302E0054686543
:10D5280020536F667444657669636520646F65731C
:10D53800206E6F7420636F6E7461696E2074686505
:10D54800206D61676963206E756D6265722069641C
:10D55800656E74696679696E6720697420617320E5
:10D568006120536F66744465766963652E0054685C
:10D578006520536F66744465766963652073697ABC
:10D588006520696E2074686520696E666F20737403
:10D598007275637420697320746F6F20736D616C8A
:10D5A8006C20636F6D7061726564207769746820A0
:10D5B8007468652073697A65207265706F72746526
:10D5C8006420696E2074686520696E697420636FD1
:10D5D8006D6D616E642E00546865206E657720530A
:10D5E8006F6674446576696365206973206F662089
:10D5F8006120646966666572656E742066616D692E
:10D608006C79207468616E20746865207072657327
:10D61800656E7420536F66744465766963652E2061
:10D62800436F6D7061746962696C697479206361B4
:10D638006E6E6F742062652067756172616E7465C5
:10D6480065642E00496E76616C69646174696E6701
:10D65800206170702062656361757365206974204C
:10D66800697320696E636F6D70617469626C65209F
:10D67800776974682074686520536F6674446576AA
:10D688006963652E004D616A6F722053442075707E
:10D698006461746520627574206E6F20424C2E2080
:10D6A80041626F727420746F2061766F69642069BB
:10D6B8006E636170616369746174696E6720746810
:10D6C8006520424C2E00426F6F742076616C69644D
:10D6D8006174696F6E206F6620626F6F746C6F6122
:10D6E800646572206973206E6F7420737570706F33
:10D6F8007274656420616E642077696C6C20626561
:10D708002069676E6F7265642E006E72665F64666C
:10D71800755F76616C69646174696F6E00433A5C29
:10D728006E5246355F53444B5F31372E302E325F91
:10D73800643637346464652D315C636F6D706F6E69
:10D74800656E74735C6C69627261726965735C6240
:10D758006F6F746C6F616465725C6466755C6E7221
:10D76800665F6466755F7665725F76616C69646131
:10D7780074696F6E2E6300496E76616C6964206609
:10D7880069726D7761726520747970652E00496ED3
:10D7980076616C6964206861736820747970652E9D
:10D7A800004E6F2048572076657273696F6E2E00A1
:10D7B8004661756C74792048572076657273696F75
:10D7C8006E2E00534420726571206E6F74206D6553
:10D7D800742E006861735F66775F76657273696F30
:10D7E8006E2069732025730D0A00735F6466755F88
:10D7F80073657474696E67732E6170705F76657295
:10D8080073696F6E2069732025730D0A002D2D2D05
:10D818002D2D2D2D2D2D2D2D322D2D2D2D2D2D2D2B
:10D828002D2D2D2D2D0D0A002D2D2D2D2D2D2D2D90
:10D838002D2D2D332D2D2D2D2D2D2D2D2D2D2D2D0A
:10D848000D0A002D2D2D2D2D2D2D2D2D2D2D342D69
:10D858002D2D2D2D2D2D2D2D2D2D2D0D0A0046571D
:10D868002076657273696F6E20746F6F206C6F77A6
:10D878002E0046572076657273696F6E206D697346
:10D8880073696E672E006E72665F6466755F766593
:10D89800725F76616C69646174696F6E006E72663E
:10D8A8005F7364680001000007000000E8A6070035
:10D8B800F0A6070008000000F8A6070008A7070060
:10D8C80008000000F0A60700F8A6070008000000FE
:10D8D80073645F626C655F6366675F73657428294C
:10D8E8002072657475726E6564202573207768658B
:10D8F8006E20617474656D7074696E6720746F2032
:10D9080073657420424C455F434F4E4E5F43464714
:10D918005F4741502E0073645F626C655F636667A2
:10D928005F73657428292072657475726E6564204A
:10D938002573207768656E20617474656D707469ED
:10D948006E6720746F2073657420424C455F4741B1
:10D95800505F4346475F524F4C455F434F554E54C7
:10D968002E0073645F626C655F6366675F736574DE
:10D9780028292072657475726E6564202573207776
:10D9880068656E20617474656D7074696E67207463
:10D998006F2073657420424C455F434F4E4E5F4382
:10D9A80046475F474154542E0073645F626C655F5D
:10D9B8006366675F73657428292072657475726E73
:10D9C8006564202573207768656E20617474656DC1
:10D9D8007074696E6720746F2073657420424C45BB
:10D9E8005F434F4D4D4F4E5F4346475F56535F551C
:10D9F8005549442E0073645F626C655F6366675FB8
:10DA080073657428292072657475726E65642025A3
:10DA180073207768656E20617474656D7074696EC3
:10DA28006720746F2073657420424C455F474154EA
:10DA380054535F4346475F415454525F5441425FD9
:10DA480053495A452E0073645F626C655F6366676D
:10DA58005F73657428292072657475726E65642019
:10DA68002573207768656E20617474656D707469BC
:10DA78006E6720746F2073657420424C455F474180
:10DA88005454535F4346475F534552564943455F95
:10DA98004348414E4745442E00496E737566666992
:10DAA8006369656E742052414D20616C6C6F6361CF
:10DAB80074656420666F722074686520536F66749D
:10DAC8004465766963652E004368616E67652074F6
:10DAD80068652052414D207374617274206C6F63C5
:10DAE8006174696F6E2066726F6D203078257820BA
:10DAF800746F20307825782E004D6178696D756DCA
:10DB08002052414D2073697A6520666F72206170DA
:10DB1800706C69636174696F6E2069732030782551
:10DB2800782E0073645F626C655F656E61626C6518
:10DB380028292072657475726E65642025732E001D
:10DB48006E72665F7364685F626C6500E0A60700CA
:10DB5800E8A60700080000006E72665F7364685FDD
:10DB6800736F630008A7070010A7070008000000EC
:10DB780043000000504F5349580000002020202047
:10DB88002020202020682828282820202020202025
:10DB98002020202020202020202020204810101085
:10DBA800101010101010101010101010848484849D
:10DBB8008484848484841010101010101081818152
:10DBC80081818101010101010101010101010101BD
:10DBD8000101010101010110101010101082828250
:10DBE800828282020202020202020202020202028D
:10DBF8000202020202020210101010200007032085
:10DC080004170201085710408000000078DB070065
:10DC18007CDC070090DD070053756E004D6F6E00C9
:10DC2800547565005765640054687500467269004C
:10DC380053617400000000004A616E00466562008E
:10DC48004D617200417072004D6179004A756E0035
:10DC58004A756C0041756700536570004F63740026
:10DC68004E6F76004465630000000000414D00508F
:10DC78004D000000B4DD0700B0DD0700B0DD07008F
:10DC8800B0DD0700B0DD0700B0DD0700B0DD07003C
:10DC9800B0DD0700B0DD0700B0DD0700FFFFFFFFC4
:10DCA800FFFFFFFFFFFFFFFFFFFF0000F0DC0700A3
:10DCB80020DC07002CDD070040DC070074DC0700CF
:10DCC800D4DC070084DD0700E0DC0700256D2F2584
:10DCD800642F257900000000256120256220256534
:10DCE800202554202559000053756E646179004D34
:10DCF8006F6E646179005475657364617900576566
:10DD0800646E6573646179005468757273646179CF
:10DD1800004672696461790053617475726461794F
:10DD2800000000004A616E75617279004665627292
:10DD380075617279004D6172636800417072696C37
:10DD4800004D6179004A756E65004A756C7900412D
:10DD580075677573740053657074656D62657200DC
:10DD68004F63746F626572004E6F76656D6265729F
:10DD780000446563656D62657200000025483A25B8
:10DD88004D3A255300000000A1A30700BDA30700DA
:10DD9800C9A30700D5A30700F1A30700FDA3070047
:0EDDA80009A4070017A40700000000002E00C9
:10DDB80000000000FF00000000000000000000005C
:10DDC800000000000000000000000000000000004B
:10DDD8000000000001000000182B0020282B002064
:10DDE8000090D003FF00FFFF0100000000E00700E3
:10DDF80014DC070014DC070014DC070014DC07003F
:04DE080014DC07001F
:020000020000FC
:020000041000EA
:0410140000200700B1
:0410180000E00700ED
:040000037000235D09
:00000001FF
